:020000040800F2
:10000000C80B0020E10300089D0100089F010008C3
:10001000A3010008A7010008AB01000800000000D0
:10002000000000000000000000000000AF01000818
:10003000B101000800000000B3010008B50100088C
:10004000FB030008FB030008FB030008FB03000898
:10005000FB030008FB030008FB030008FB03000888
:10006000FB030008FB030008FB030008FB03000878
:10007000FB030008FB030008FB030008FB03000868
:10008000FB030008FB030008FB030008FB03000858
:10009000FB030008FB030008FB030008FB03000848
:1000A000FB030008FB030008FB030008FB03000838
:1000B0000D2C0008FB030008F52B0008FB030008CB
:1000C000FB030008FB030008FB030008FB03000818
:1000D000FB030008FB030008FB030008FB03000808
:1000E0000F340008FB030008FB03000800F002F8CF
:1000F00000F03FF80AA090E8000C82448344AAF183
:100100000107DA4501D100F034F8AFF2090EBAE880
:100110000F0013F0010F18BFFB1A43F0010318473B
:10012000C0980000E0980000103A24BF78C878C159
:10013000FAD8520724BF30C830C144BF04680C60ED
:10014000704700000023002400250026103A28BF35
:1001500078C1FBD8520728BF30C148BF0B60704739
:10016000642906F0EB83002070471FB51FBD10B552
:1001700010BD06F0A3FD1146FFF7F7FF00F00CF9E4
:1001800006F0C1FD03B4FFF7F2FF03BC02F066F90D
:1001900030BF72B662B680F308887047704700BF00
:1001A000FEE700BFFEE700BFFEE700BFFEE77047C7
:1001B00070477047704700000CB500200190009018
:1001C0006C48006840F480306A49086000BF6948A4
:1001D000006800F4003000900198401C01900098E5
:1001E00018B90198B0F5A06FF1D16248006800F429
:1001F000003010B10120009001E000200090009834
:10020000012843D15C48006840F010005A4908605A
:100210000846006820F0030008600846006840F0C7
:1002200002000860534840685249486008464068E8
:1002300048600846406840F480604860084640686E
:1002400020F47C1048600846406840F4E81048609C
:100250000846006840F08070086000BF45480068AC
:1002600000F000700028F9D04248406820F00300F8
:10027000404948600846406840F00200486000BFBE
:100280003C48406800F00C000828F9D10CBD10B5BE
:10029000FFF792FF10BD10B53648006840F001002E
:1002A000344908600846406834490840314948608C
:1002B00008460068324908402E4908600846006830
:1002C00020F4802008600846406820F4FE00486062
:1002D0004FF41F008860FFF7DAFF4FF000602949F4
:1002E000086010BD10B5002100200022214B5B6882
:1002F00003F00C0121B1042906D0082928D107E018
:10030000214B224C236027E01F4B204C236023E02D
:10031000184B5B6803F47010164B5B6803F4803273
:10032000022303EB904022B9194B4343174C23603F
:100330000DE0104B5B6803F4003323B1144B4343CF
:10034000124C236003E0104B4343104C236003E046
:100350000D4B0E4C236000BF00BF064B5B68C3F320
:1003600003130C4CE15C094B1B68CB40074C23602A
:1003700010BD000000100240002002400000FFF805
:10038000FFFFF6FE08ED00E000127A0000000020FA
:1003900000093D0004000020022001F007FF01F0E9
:1003A00095FE022001F0ECFF012001F0E9FF02F0D0
:1003B000A7F8002141F61F4002F008FB02F05EFBA7
:1003C00002F0A9FB02F036FC02F037FA06F033F92E
:1003D00006F045F902F0C2FE01E003F0A3F8FCE7E5
:1003E0000948804709480047FEE7FEE7FEE7FEE7C9
:1003F000FEE7FEE7FEE7FEE7FEE7FEE70448054905
:10040000054A064B7047000097020008ED000008FF
:10041000C8050020C80B0020C8070020C80700201E
:1004200031490143314A1160704770B50021002302
:100430000F22C47804B32D4C246804F4E064C4F59E
:10044000E064210AC1F10403CA40447804FA03F1CC
:100450008478144021430901254C0678A15504787D
:1004600004F01F050124AC4005786D11AD0005F1C5
:10047000E025C5F8004109E0047804F01F050124D7
:10048000AC401C4D0678761145F8264070BD1A4ADE
:100490000A400243154B1B1F1A60704739B1134ABB
:1004A000121D12680243114B1B1D1A6006E00F4A11
:1004B000121D126882430D4B1B1D1A6070470428E1
:1004C00008D14FF0E021096941F004014FF0E0222A
:1004D000116107E04FF0E021096921F004014FF0BC
:1004E000E0221161704700000000FA050CED00E009
:1004F00000E400E080E100E080FFFF1F10B5012074
:1005000000F0A2FC002000F09FFC10BD2A4908600A
:1005100070472949091F08607047274984310860DE
:10052000704701460020254A10884FF67F42104050
:100530000843224A10807047014600201F4A108855
:100540004FF68072104008431C4A1080704708B56F
:1005500000220092194A2C3A0092009A024400921A
:10056000009A116008BD08B50146002000901348AC
:100570002C3800900098084400900098008808BD2E
:100580000D489C300068C0B270470C4808300088A5
:1005900040F0010009490831088070470648A03042
:1005A0000068C0B2704705480830008840F002007B
:1005B000024908310880704704860D422C6C0040C7
:1005C000002044490860091D0860091D0860091DD4
:1005D000086041483F4914310860704700213D4997
:1005E0008279002A3AD00A46126803689A430B4679
:1005F0001A600A1D126803689A430B1D1A6002797B
:1006000011440A6803681A430A60324A08321268C1
:1006100003689A432F4B08331A601A1D1268036847
:100620009A432C4B0C331A604279102A0ED11A1FB0
:10063000126803681A43274B08331A601A1D1268A0
:1006400003681A43234B0C331A600DE021494279A9
:1006500011440A6803681A430A6005E002791144EC
:100660000A6803689A430A607047002101600171BB
:100670000C214171002181717047164910310968C0
:100680000143144A10321160704701460020114A9C
:10069000143212680A400AB1012000E000207047BD
:1006A0000C49143108607047014600200022094BB4
:1006B0001B6803EA0102074B14331B680B4013B19C
:1006C0000AB1012000E0002070470249143108609F
:1006D0007047000000040140FFFF0F0010B5044602
:1006E000CC48844208D10121042000F093FB002172
:1006F000042000F08FFB46E0C748844208D1012166
:10070000082000F087FB0021082000F083FB3AE07E
:10071000C248844208D10121102000F07BFB002157
:10072000102000F077FB2EE0BD48844208D1012163
:10073000202000F06FFB0021202000F06BFB22E066
:10074000B848844208D10121402000F063FB002119
:10075000402000F05FFB16E0B348844208D101213D
:10076000802000F057FB0021802000F053FB0AE0BE
:10077000AE48844207D10121801500F04BFB0021D7
:10078000A01500F047FB10BD10B50121084600F090
:1007900041FB0021012000F03DFB10BD2DE9F0419F
:1007A000024600250026002000230024002791F89F
:1007B00003C00CF00F0591F803C00CF0100CBCF155
:1007C000000F03D091F802C04CEA050591F800C073
:1007D000BCF1000F31D0146800202BE04FF0010C69
:1007E0000CFA00F3B1F800C00CEA03069E4220D1D7
:1007F00083004FF00F0C0CFA03F7BC4305FA03FC1F
:100800004CEA040491F803C0BCF1280F06D14FF064
:10081000010C0CFA00FCC2F814C00AE091F803C005
:10082000BCF1480F05D14FF0010C0CFA00FCC2F8E6
:1008300010C0401C0828D1D31460B1F800C0BCF12E
:10084000FF0F34DD546800202EE000F1080C4FF05B
:10085000010808FA0CF3B1F800C00CEA03069E4246
:1008600021D183004FF00F0C0CFA03F7BC4305FABB
:1008700003FC4CEA040491F803C0BCF1280F05D135
:1008800000F1080C08FA0CF8C2F8148091F803C0C3
:10089000BCF1480F07D100F1080C4FF0010808FA2D
:1008A0000CF8C2F81080401C0828CED35460BDE874
:1008B000F0814FF6FF710180022181700421C17027
:1008C00070470246002093680B400BB1012000E006
:1008D000002070470146886880B2704702460020B9
:1008E000D3680B400BB1012000E0002070470146A7
:1008F000C86880B2704701617047416170470AB1B2
:10090000016100E041617047C16070474FF480327F
:100910000A4382618161826182698269704702460D
:100920000020434B18684FF68073184040EA0210CD
:1009300008433F4B186070473E49C8617047F0B5A7
:100940000A46002300240021002500F00046B6F1ED
:10095000004F02D1364EF16901E0354E7168C0F3A7
:10096000034583B200F44016B6F5401F08D121F0CC
:1009700070612F4E766826F070662D4F7E6012E013
:1009800000F48016B6F5801F06D1032606FA05F49A
:10099000A14341F0706106E0460D360103FA06F608
:1009A000B14341F0706122B1460D360103FA06F6FB
:1009B000314300F00046B6F1004F02D11C4EF16108
:1009C00001E01B4E7160F0BD30B500228B071C0F9B
:1009D0000F2303FA04F2164B08338C1053F824301B
:1009E0009343134C08348D1044F8253023468C1063
:1009F00053F824308C07240F00FA04F423430C4CE2
:100A000008348D1044F8253030BD0A49DC310860C7
:100A10007047000000080140000C01400010014038
:100A20000014014000180140001C0140002001405A
:100A3000000001400000204210B50121080700F02D
:100A4000F6F900214FF0805000F0F1F910BD2A496D
:100A50000862704728490861704701460020274A0C
:100A6000106820F0E0000843106070472249A03170
:100A70000860704710B502460020204B186820F02F
:100A80000300104318601E4B1B6843F004031C4C0A
:100A90002360012901D130BF00E020BF184B1B6843
:100AA00023F00403164C236010BD1448006840F086
:100AB0000400124908600846006840F0020008601F
:100AC0000F48006840F004000D49086000BF00BFF7
:100AD00030BF704701460020084A52680A400AB1F8
:100AE000012000E0002070470449096841EA8001C4
:100AF000024A11607047000000000E420070004082
:100B000010ED00E0DF48006840F00100DD490860BA
:100B100008464068DC490840DA49486008460068F1
:100B2000DA490840D74908600846006820F4802068
:100B300008600846406820F4FE0048604FF41F003B
:100B400088607047CF49096821F48031CD4A11602F
:100B50001146096821F480211160B0F5803F03D06F
:100B6000B0F5802F0ED106E0C649096841F4803106
:100B7000C44A116007E0C349096841F4A021C14A91
:100B8000116000E000BF00BF704710B501460022B1
:100B9000002300204A11012A02D1BA4C236806E042
:100BA000022A02D1B74C236A01E0B64C636A01F015
:100BB0001F02012494401C400CB1012000E00020E1
:100BC00010BD38B5002000900024002500BF312062
:100BD000FFF7DBFF05460098401C00900098B0F539
:100BE000A06F01D0002DF2D03120FFF7CEFF08B169
:100BF000012400E00024204638BD01460020A14A1F
:100C0000106820F0F80040EAC10010607047A04969
:100C100008607047024600209A4B586820F47C1008
:100C200042EA01031843974B586070479849086699
:100C3000704701460020934A506820F003000843A3
:100C4000506070478F48406800F00C0070470146C4
:100C500000208C4A506820F0F00008435060704734
:100C600001460020874A506820F4E0600843506045
:100C7000704701460020834A506820F4605040EAE3
:100C8000C1005060704729B17E4A527A02437D4BC1
:100C90005A7204E07B4A527A82437A4B5A72704706
:100CA0007B49D8310860704701460020754A50687A
:100CB00020F440400843506070470021714A2032C0
:100CC0001170704A82F82010012802D004280AD13D
:100CD00004E001216B4A2032117005E00521694AC8
:100CE0002032117000E000BF00BF70476949086002
:100CF00070476449096A0143624A11627047654955
:100D000044390860704730B50021002200240023D8
:100D10005C4D6D6805F00C0121B1042905D008294E
:100D200023D105E05C4D056022E05B4D05601FE0CE
:100D3000544D6D6805F47012524D6D6805F48034A1
:100D4000022505EB92421CB9544D554305600BE05A
:100D50004C4D6D6805F400351DB1504D554305608F
:100D600002E04D4D5543056002E04B4D056000BF6C
:100D700000BF444D6D6805F0F0010909484D6B5CFA
:100D80000568DD4045603F4D6D6805F4E061090A86
:100D9000434D6B5C4568DD4085603A4D6D6805F4F8
:100DA0006051C90A3E4D6B5C4568DD40C560354DFC
:100DB0006D6805F44041890B3A4D6B5CC568B5FB25
:100DC000F3F5056130BD29B12E4A526902432D4B1E
:100DD0005A6104E02B4A526982432A4B5A61704798
:100DE00029B1284A92690243264B9A6104E0254AB8
:100DF00092698243234B9A61704729B1214AD26993
:100E00000243204BDA6104E01E4AD26982431D4B43
:100E1000DA61704729B11B4AD2680243194BDA6084
:100E200004E0184AD2688243164BDA60704729B151
:100E3000144A12690243134B1A6104E0114A126901
:100E40008243104B1A61704712494039086070475D
:100E50000F49C86470470B49C87170470948406A18
:100E600040F0807007494862704701460020054AFB
:100E700092680A400AB1012000E000207047014951
:100E800088727047001002400000FFF8FFFFF6FE76
:100E9000000042428004424200127A0000093D00F4
:100EA000280000203800002010B50446FE48844287
:100EB00008D10121C014FFF7ADFF0021E014FFF7B6
:100EC000A9FFC4E0B4F1804F08D101210846FFF723
:100ED000AEFF00210120FFF7AAFFB8E0F3488442EB
:100EE00008D101210220FFF7A2FF00210220FFF715
:100EF0009EFFACE0EE48844208D101210420FFF7B8
:100F000096FF00210420FFF792FFA0E0E948844209
:100F100008D101210820FFF78AFF00210820FFF7F0
:100F200086FF94E0E448844208D101211020FFF7B5
:100F30007EFF00211020FFF77AFF88E0DF4884421F
:100F400008D101212020FFF772FF00212020FFF7A8
:100F50006EFF7CE0DA48844208D101214014FFF79B
:100F600059FF00216014FFF755FF70E0D548844217
:100F700009D10121C804FFF74DFF00214FF40020E3
:100F8000FFF748FF63E0D048844209D101210805FA
:100F9000FFF740FF00214FF48010FFF73BFF56E0C2
:100FA000CA48844209D101214805FFF733FF0021D7
:100FB0004FF40010FFF72EFF49E0C548844208D1E6
:100FC00001214020FFF733FF00214020FFF72FFFD2
:100FD0003DE0C048844208D101218020FFF727FF6F
:100FE00000218020FFF723FF31E0BB48844208D175
:100FF00001218015FFF71BFF0021A015FFF717FF48
:1010000025E0B648844209D101210804FFF702FF18
:1010100000214FF48030FFF7FDFE18E0B048844215
:1010200009D101214804FFF7F5FE00214FF40030FB
:10103000FFF7F0FE0BE0AB48844208D101218804A1
:10104000FFF7E8FE00214FF48020FFF7E3FE10BD1C
:1010500000220288944B98420ED0994B98420BD0B4
:10106000B0F1804F08D0914B984205D0904B9842F8
:1010700002D0904B984204D14FF68F731A404B88A0
:101080001A438D4B984207D08C4B984204D04FF6B0
:10109000FF431A40CB881A4302808B8883850B88D4
:1010A0000385814B98420BD0854B984208D08B4BDF
:1010B000984205D08A4B984202D08A4B984201D17F
:1010C0000B7A038601238382704770B500240022C7
:1010D0000023058C4FF6FE7635400584028C83880C
:1010E000048B4FF68F752C40B51E2C400D882C4379
:1010F000751E2A400D892A434D882A436A4DA8420D
:101100000BD06F4DA84208D0744DA84205D0744D45
:10111000A84202D0734DA84213D14FF6F7752A406A
:101120004D892A434FF6FB752A408D882A434FF696
:10113000FF652B404FF6FF552B408D892B43CD8902
:101140002B4383800483CD888586028470BD70B56F
:10115000002400220023058C4FF6EF7635400584ED
:10116000028C8388048B48F6FF752C404FF6FF45B0
:101170002C400D884FF6FF7606EA05252C434FF6E6
:10118000DF752A400D8906EA05152A434D8806EACF
:1011900005152A43444DA84202D0494DA8421DD10D
:1011A0004FF67F752A404D894FF6FF7606EA051502
:1011B0002A434FF6BF752A408D8806EA05152A4353
:1011C0004FF6FF352B404FF2FF752B408D8906EA15
:1011D00085052B43CD8906EA85052B43838004834F
:1011E000CD880587028470BD70B5002400220023DD
:1011F000058C4FF6FF6635400584028C8388848B0E
:101200004FF68F752C404FF6FC752C400D882C4303
:101210004FF6FF552A400D894FF6FF7606EA052561
:101220002A434D8806EA05252A431F4DA84202D0CD
:10123000234DA8421DD14FF2FF752A404D894FF62C
:10124000FF7606EA05252A434FF6FF352A408D88AA
:1012500006EA05252A434EF6FF752B404DF6FF752D
:101260002B408D8906EA05152B43CD8906EA051525
:101270002B4383808483CD888587028470BD70B5BD
:10128000002200230024058C4EF6FF7635400584AD
:10129000038C8488828B48F6FF752A404FF6FF4501
:1012A0002A400D8820E00000002C0140000400408E
:1012B00000080040000C00400010004000140040F6
:1012C00000340140004C01400050014000540140F6
:1012D00000180040001C0040002000400040014079
:1012E00000440140004801404FF6FF7606EA05251C
:1012F0002A434DF6FF752B400D8906EA05352B4331
:101300004D8806EA05352B43FA4DA84202D0FA4D26
:10131000A84208D14BF6FF752C408D894FF6FF7619
:1013200006EA85152C4384808283CD88A0F840503E
:10133000038470BD828B4FF2FF331A408283828B0D
:101340004FF6FF7303EA01231A4382837047F0B517
:101350000C461546002200210026078C4EF6FF7C25
:1013600007EA0C070784828B018C4FF6FF7707EAA8
:10137000043640F6FF473A404FF6FF7707EA052765
:101380003A434FF6FF7707EA03373A43D94FB8425B
:101390000ED0D94FB8420BD0B0F1804F08D0D74F04
:1013A000B84205D0D64FB84202D0D64FB84206D187
:1013B0004DF6FF77394046F48057394305E047F64C
:1013C000FF57394044F48057394382830184F0BD8C
:1013D000828B4FF6F3731A408283828B0A43828397
:1013E0007047F0B50C461546002200210026078CF8
:1013F0004FF6FF6C07EA0C070784828B018C4FF6CF
:10140000FF7707EA04264FF60C773A404FF6FF774E
:1014100007EA03172F433A43B64FB8420ED0B64FF0
:10142000B8420BD0B0F1804F08D0B44FB84205D0CD
:10143000B34FB84202D0B34FB84206D14FF6FF5770
:10144000394046F48077394305E04FF2FF57394081
:1014500044F48077394382830184F0BD028B4FF2DC
:10146000FF331A400283028B4FF6FF7303EA012316
:101470001A4302837047F0B50C461546002200213E
:101480000026078C4FF6EF7C07EA0C070784028BD7
:10149000018C4FF6FF7707EA041640F6FF473A4003
:1014A0004FF6FF7707EA03373A434FF6FF7707EA2D
:1014B00005273A438F4FB8420ED08F4FB8420BD01A
:1014C000B0F1804F08D08D4FB84205D08C4FB84254
:1014D00002D08C4FB84206D14FF6DF77394046F044
:1014E0001007394305E04FF65F77394044F01007A5
:1014F000394302830184F0BD028B4FF6F3731A4027
:101500000283028B0A4302837047F0B50C461546EE
:1015100000220021068C4FF6FE773E400684028BA7
:10152000018C4FF60C7632407E1C06EA03162E43E1
:101530003243704EB0420ED06F4EB0420BD0B0F17D
:10154000804F08D06D4EB04205D06D4EB04202D0F3
:101550006C4EB04206D14FF6FD76314044F00106A4
:10156000314305E04FF6F576314044F00106314352
:1015700002830184F0BD70B505460C465D48854286
:101580000ED05D4885420BD0B5F1804F08D05B4846
:10159000854205D05A48854202D05A48854200D13A
:1015A00000E000BF208850B92389A28861882846BE
:1015B000FFF7ABFFE1882846FFF79EFF25E0208874
:1015C00004280AD12389A28861882846FFF753FF9F
:1015D000E1882846FFF742FF17E0208808280AD153
:1015E0002389A28861882846FFF7FBFEE188284608
:1015F000FFF7EEFE09E02389A28861882846FFF7FD
:10160000A6FEE1882846FFF795FE70BD2DE9F04162
:1016100005460C4600260127608808B9022600E02E
:101620000026A088012801D1022700E00127208898
:10163000A0B92389A28861882846FFF766FFE18860
:101640002846FFF759FF23893A4631462846FFF7D7
:1016500012FFE1882846FFF701FF13E02389A288E3
:1016600061882846FFF707FFE1882846FFF7F6FE66
:1016700023893A4631462846FFF747FFE188284646
:10168000FFF73AFFBDE8F0810A884B881A438B8840
:101690001A43CB881A430B891A434B891A438B8907
:1016A0001A43A0F8442070474FF6FF718180002153
:1016B0000180C1804180017270470021018041801A
:1016C0008180C180018141818181C1817047002178
:1016D00001804180012181800021C180018170470A
:1016E0000021018041808180C1800181418181810F
:1016F00070470000002C014000340140000400400D
:1017000000080040000C004021B1028842F00102B4
:10171000028004E002884FF6FE731A400280704790
:1017200031B1B0F8442042F40042A0F8442005E072
:10173000B0F84420C2F30E02A0F8442070471AB15A
:1017400083890B43838102E083898B4383817047C4
:101750008182704741EA0203A0F8483070471AB10D
:1017600083890B43838102E083898B4383817047A4
:1017700001894FF6F8721140018170470A46002135
:1017800001894FF68F73194011430181704730B5BD
:1017900004460D4629462046FFF7F0FF208940F019
:1017A0000700208130BD2DE9F04104460D46164664
:1017B0001F46602D06D13B46012231462046FFF7E9
:1017C0005AFE05E03B46012231462046FFF79DFECA
:1017D00029462046FFF7D2FF208940F007002081EC
:1017E000BDE8F08130B50C4600210189C9B24FF641
:1017F000FF7505EA0325154325432943018130BDC3
:101800002DE9F04105460E4617469846002443460A
:101810003A4631462846FFF7E5FF2C894FF6F87027
:10182000044044F007044FF68F70044044F0700405
:101830002C81BDE8F081F0B504460D4616461F46E2
:101840003B46324629462046FFF7CCFF208940F42C
:1018500080402081F0BD0185828270470A460021C8
:1018600001884FF68F731940114301807047F0B51E
:101870000C4615461E460021002200230189028BDA
:10188000038C4FF6F877394021434FF6FC473A4036
:1018900040F201173A434FF6DD773B404FF6FF77B2
:1018A00007EA06172F433B43018102830384F0BDFF
:1018B0000A460021018B4FF68F73194011430183B3
:1018C00070470A460021018B48F6FF7319404FF616
:1018D000FF7303EA02231943018370470A4600217C
:1018E000818B4FF68F7319401143818370470A46ED
:1018F0000021818B48F6FF7319404FF6FF7303EA0E
:10190000022319438183704721B1028842F080028B
:10191000028004E002884FF67F731A40028070470D
:1019200021B1828842F00402828004E082884FF66E
:10193000FB731A408280704721B1828842F008020E
:10194000828004E082884FF6F7731A4082807047E5
:1019500021B1828842F00102828004E082884FF641
:10196000FE731A40828070470A460021018B4FF6B1
:10197000F77319401143018370470A460021018B18
:101980004FF2FF7319404FF6FF7303EA0223194326
:10199000018370470A460021818B4FF6F773194087
:1019A0001143818370470A460021818B4FF2FF73F8
:1019B00019404FF6FF7303EA0223194381837047EE
:1019C0000A460021018B4FF6FB7319401143018336
:1019D00070470A460021018B4FF6FF3319404FF63E
:1019E000FF7303EA02231943018370470A4600216B
:1019F000818B4FF6FB7319401143818370470A4670
:101A00000021818B4FF6FF3319404FF6FF7303EA35
:101A100002231943818370470A460021018B4FF648
:101A20007F7319401143018370470A460021018BDF
:101A3000C1F30E014FF6FF7303EA0223194301833A
:101A400070470A460021818B4FF67F73194011437E
:101A5000818370470A460021818BC1F30E014FF646
:101A6000FF7303EA02231943818370470A4600216A
:101A7000018C4FF6FD7319401143018470470A46EB
:101A80000021018C4FF6F773194011430184704710
:101A90000A460021018C4FF6DF7319404FF6FF73A1
:101AA00003EA02131943018470470A460021018C9E
:101AB0004FF67F7319404FF6FF7303EA0213194381
:101AC000018470470A460021018C4FF6FF531940EC
:101AD0004FF6FF7303EA02231943018470470A4655
:101AE0000021018C4FF2FF7319404FF6FF7303EA98
:101AF00002231943018470470A460021018C4DF6E8
:101B0000FF7319404FF6FF7303EA02331943018450
:101B1000704730B5002301248C40A3B2048C9C4351
:101B20000484048C02FA01F5ADB22C43048430BD68
:101B300030B5002304248C40A3B2048C9C4304845D
:101B4000048C02FA01F5ADB22C43048430BD70B5AB
:101B50000346002000241846183001258D40ACB201
:101B60001D8CA5431D8409B1082909D100EB610032
:101B7000056825F0700505600568154305600EE0F1
:101B80000D1FC5F34E052844056825F4E0450560A2
:101B900005684FF6FF7606EA02263543056070BDFC
:101BA00021B1028842F00202028004E002884FF66E
:101BB000FD731A400280704721B1028842F004028E
:101BC000028004E002884FF6FB731A4002807047DF
:101BD00021B1828842F08002828004E082884FF640
:101BE0007F731A408280704702884FF6F7731A405D
:101BF000028002880A430280704782884FF68F7302
:101C00001A40828082880A438280704702894FF698
:101C1000F8731A40028102890A43028170470289DF
:101C20004FF67F731A40028102890A43028170478E
:101C3000818470478185704781867047018770472E
:101C400081877047A0F84010704702884FF6FF4325
:101C50001A40028002880A43028070470146888E3B
:101C600070470146088F70470146888F70470146CC
:101C7000B1F8400070470146888C70470146088DD6
:101C8000704702460020138A0B400BB1012000E090
:101C900000207047CA430282704730B502460020D8
:101CA00000230024158A05EA0103958905EA010449
:101CB00013B10CB1012000E0002030BDCA43028204
:101CC0007047000010B50446FB48844209D1012149
:101CD0008803FFF79FF800214FF48040FFF79AF840
:101CE00032E0F648844209D101214804FFF79FF809
:101CF00000214FF40030FFF79AF825E0F0488442C5
:101D000009D101218804FFF792F800214FF48020C7
:101D1000FFF78DF818E0EB48844209D10121C8048F
:101D2000FFF785F800214FF40020FFF780F80BE063
:101D3000E548844208D101210805FFF778F8002121
:101D40004FF48010FFF773F810BD2DE9F04786B00F
:101D500005460E460024A24600BFA1460027B089D2
:101D600000B100BF2F462C8A4CF6FF700440F0886B
:101D700004432C82AC894EF6F3100440B0883189BC
:101D80000843718908430443AC81AC8A4FF6FF4095
:101D90000440B0890443AC8201A8FEF7B4FFC648F2
:101DA000874202D1DDF810A001E0DDF80CA0A8897F
:101DB00000F4004040B10AEBCA0000EB0A103168A1
:101DC0004900B0FBF1F807E00AEBCA0000EB0A108B
:101DD00031688900B0FBF1F86420B8FBF0F0040131
:101DE0002009642101FB1089A88900F4004040B15A
:101DF000322000EBC900B0FBF1F000F00700044313
:101E000008E0322000EB09106421B0FBF1F000F093
:101E10000F0004432C8106B0BDE8F0874FF4165143
:101E2000016000218180C18001810C21418100215C
:101E30008181704710B502460020108A4FF2FF03DF
:101E400018400B884C8823438C882343CC88234339
:101E50001843108210BD0021018041808180C18023
:101E6000704721B1828942F40052828104E0828964
:101E70004DF6FF731A4082817047F0B50346002487
:101E800000260025002040F66A17B94200D100BFA5
:101E90001846C1F3421401F01F06012707FA06F5A0
:101EA000012C01D10C3004E0022C01D1103000E0F3
:101EB00014301AB107682F43076002E00768AF4388
:101EC0000760F0BD1AB1838A0B43838202E0838AE4
:101ED0008B4383827047028A4FF6F0731A40028266
:101EE000028A0A430282704782894FF2FF731A40C6
:101EF000828182890A438281704721B1828942F0BE
:101F00000202828104E082894FF6FD731A408281C9
:101F10007047028A4FF6DF731A400282028A0A4330
:101F20000282704721B1028A42F48042028204E0B8
:101F3000028A4BF6FF731A4002827047C1F308020F
:101F40008280704701468888C0F308007047818905
:101F500041F0010181817047028BD2B20283028B72
:101F600042EA012202837047028B02F47F4202831D
:101F7000028B0A430283704721B1828A42F0200219
:101F8000828204E0828A4FF6DF731A4082827047B1
:101F900021B1828A42F01002828204E0828A4FF6E6
:101FA000EF731A408282704721B1828A42F00802A0
:101FB000828204E0828A4FF6F7731A408282704769
:101FC00021B1828942F40042828103E08289C2F316
:101FD0000E028281704721B1828A42F400628282BD
:101FE00004E0828A4FF2FF731A4082827047828A2D
:101FF0004FF6FB731A408282828A0A4382827047BC
:1020000021B1828A42F00202828204E0828A4FF683
:10201000FD731A408282704702460020B1F5007FAE
:1020200000D100BF13880B400BB1012000E000205D
:10203000704701F40072B2F5007F00D100BFCA43BF
:102040000280704770B5024600240023002500205E
:1020500040F66A16B14200D100BFC1F3421501F04B
:102060001F03012606FA03F3012D02D1968933409E
:1020700006E0022D02D1168A334001E0968A3340F1
:102080000C12012606FA04F41688344013B10CB180
:10209000012000E0002070BD10B50022002340F6B2
:1020A0006A14A14200D100BF0A1201249440A3B2D5
:1020B000DC43048010BD00000038014000440040B3
:1020C00000480040004C00400050004010B56FF048
:1020D0000400FEF7F4F92E4800682E49B0FBF1F039
:1020E0002D4908700846007800EB4001C1EBC01094
:1020F0004FF6FF7101EAC0002849088010BD014673
:10210000254A12784A434FF0E0235A6100229A612F
:102110001A46126942F001021A6100BF4FF0E02234
:10212000106900F001021AB100F48032002AF5D0E3
:102130004FF0E022126922F001024FF0E0231A6111
:1021400000229A6170470146144A12884A434FF0B0
:10215000E0235A6100229A611A46126942F0010294
:102160001A6100BF4FF0E022106900F001021AB1BD
:1021700000F48032002AF5D04FF0E022126922F0FC
:1021800001024FF0E0231A6100229A6170470000BB
:102190000000002000127A003C0000203E000020D9
:1021A000A34A0A400243A34B1A6070470146072323
:1021B00023EA010212029F4B1B1D18684FF6FF0312
:1021C00018409D4B184310439A4B1B1D18607047D5
:1021D0002DE9F0410746884614461D462846FFF77C
:1021E000E5FFC5F1040007FA00F60F20284100EAD8
:1021F0000800064306F00F06E21704EBD262521104
:10220000920002F1E022D2F800212146E31704EB0C
:10221000D3635B11A4EB431C012303FA0CF31A43B1
:102220002046E31704EBD3635B119B0003F1E0232B
:10223000C3F800218148005D40EA06107F49085537
:10224000BDE8F08170B504460B46CE1701EB9676DB
:10225000C6F38700CE1701EB9676B610A1EB860683
:10226000B606350E764B9B6943F00103744EB3619D
:102270004FEAB63353F820300F26AE40B343714EC9
:1022800046F82030334653F8203004FA05F61E4352
:102290006C4B43F820606C4B1B6801268E40334327
:1022A000694E336002F0010343B1674B0C331B6886
:1022B00001268E403343644E0C36336002F0020335
:1022C00043B1614B08331E6801238B401E435E4BB4
:1022D00008331E6070BD00B5002059490861C86010
:1022E0001420486100208861C8610846006840F0F9
:1022F0000100086008464068544908405049486059
:1023000008460068524908404D4908600846006880
:1023100020F4802008600846406820F4FE004860F1
:102320000020886000214FF00060FFF739FF00BDFA
:1023300010B540480830006840F004003D490831BD
:1023400008603F48C06940F080503D49C86141483D
:10235000406840F480703F4948600846006840F09B
:10236000040008600846006840F002000860FDF7BD
:102370000FFF10BD3048001D2E49091D0860704731
:10238000014649062E4A926942F001022C4B9A619D
:102390002C4A083A526822F0E0622A4B083B5A6005
:1023A0001A4652680A435A60704730B50446002501
:1023B000FFF791FF2248006840F480302049086010
:1023C00000BF1F480068400C0028FAD04FF480601E
:1023D0001B494860A01EC4B20846406840EA8440D9
:1023E00048600846406840F4803048601A480068F9
:1023F00040F03200184908601148006840F08070D1
:102400000F49086000BF0E480068400E0028FAD04F
:102410000B48406840F002000949486005E0084860
:102420004068C0F3870505F00305022DF7D130BDE4
:1024300080FFFF1F08ED00E00000FA0500E400E067
:102440000010024008000140000401400000FFF8B5
:10245000FFFFF6FE0070004000200240014600BF72
:10246000704700BF244A128802F04002002AF9D0C7
:10247000C2B2214B1B1D1A80704710B586B00446AE
:10248000012144F20400FEF7ABFC4FF40070ADF8FC
:10249000140003208DF8160018208DF8170005A9E8
:1024A0001648FEF77BF94FF48060ADF81400042065
:1024B0008DF8170005A91148FEF770F90194002066
:1024C000ADF80800ADF80A00ADF80C00ADF810004A
:1024D0000C20ADF80E0001A90748FFF736FC0022DA
:1024E00040F225510448FFF7C8FC01210248FFF7DC
:1024F000B8FC06B010BD00000038014000080140E3
:1025000008B501210420FEF76BFC2020ADF8000087
:1025100048208DF8030069460B48FEF73FF908BDD7
:102520000A48007838B10A48006820B900200749F5
:1025300008700120704706480068012801D103494E
:1025400008700020F6E70000000801404400002069
:102550001401214210B50A461AB10123FE4C236032
:1025600002E00023FC4C2360002114E00023FB4C1C
:10257000236000F080031BB10123241F236003E0CC
:102580000023F64C241F23600123F44C23604306F0
:10259000180E4B1CD9B20829E8DB0123EE4C23604E
:1025A00010BD30B500241CE004F1B001C8B2002118
:1025B000FFF7D0FF00210846FFF7CCFF00211020D5
:1025C000FFF7C8FF002508E0E54901EBC501085DFC
:1025D0000121FFF7BFFF681CC5B2802DF4DB601C32
:1025E000C4B2082CE0DB30BD00B500218D20FFF720
:1025F000B1FF00211420FFF7ADFF0021AF20FFF74E
:10260000A9FF00BD00B500218D20FFF7A3FF002129
:102610001020FFF79FFF0021AE20FFF79BFF00BDBA
:1026200030B500240CE0002506E00020CC4901EB89
:10263000C5010855681CC5B2802DF6DB601CC4B20C
:10264000082CF0DBFFF7ADFF30BDF0B514460026D7
:102650007F2801DC3F2900DDF0BD0B46CF1701EBE1
:102660005777FF10C7F10707FAB2CF1701EB57777B
:10267000FF10A1EBC707FDB2C5F107070123BB405F
:10268000DEB24CB1B64B03EBC0039B5C3343B44F9B
:1026900007EBC007BB5408E0B14B03EBC0039B5CE6
:1026A000B343AF4F07EBC007BB5400BFD4E72DE9DE
:1026B000F04F80460C4615461E46A346A5F1200065
:1026C000C5B200273EE00C2E07D105EB4500A54919
:1026D00001EB800010F8079004E0A34800EB051020
:1026E00010F807904FF0000A26E009F0800028B1AA
:1026F00021464046099AFFF7A8FF09E0099808B962
:10270000012000E00020024621464046FFF79DFFE1
:102710004FEA49604FEA1069601CC4B2A4EB0B0099
:10272000B04205D15C4608F1010000F0FF0806E068
:102730000AF1010000F0FF0ABAF1080FD5DB00BF73
:10274000781CC7B2B742BEDBBDE8F08F10B50246B9
:10275000012000E050430B1EA1F10104E1B2F9D1C8
:1027600010BD2DE9FF4F81B0074691461E460E9DD4
:102770004FF0000A002439E0301B401EC1B20A208D
:10278000FFF7E4FFB9FBF0F00A21B0FBF1F201FB27
:102790001208BAF1000F16D1701EA04213DDB8F175
:1027A000000F0ED10120AB4605EBDB71491001FB98
:1027B00004710090C8B22B4620220299FFF777FFE0
:1027C00012E04FF0010A0120AB4605EBDB71491026
:1027D00001FB04710090C8B208F13001CAB22B4667
:1027E0000299FFF764FF00BF601CC4B2B442C3DBB0
:1027F00005B0BDE8F08F78B505460E46144618E0E2
:102800007A2D03DD002506F11000C6B23A2E04DD54
:10281000002005460646FFF703FF012000902278BE
:102820000C2331462846FFF742FF05F10800C5B2E8
:10283000641C20780028E3D178BD08B50121082068
:10284000FEF7CEFA3820ADF8000010208DF8030016
:1028500002208DF8020069464448FDF79FFF0121E0
:102860000420FEF7BDFA4FF40040ADF8000002204E
:102870008DF8020010208DF8030069463C48FDF7F2
:102880008DFF0120FEF7E3F80020FEF716FA002086
:10289000FDF73FFE0020FEF7DAF800202F49083947
:1028A00008606420FFF74FFC01203249C1F88C0119
:1028B0000021AE20FFF74EFE0021D520FFF74AFE93
:1028C00000215020FFF746FE0021A820FFF742FE1E
:1028D00000213F20FFF73EFE0021D320FFF73AFE04
:1028E00000210846FFF736FE00214020FFF732FEA8
:1028F00000218D20FFF72EFE00211420FFF72AFE75
:1029000000212020FFF726FE00210220FFF722FEF3
:102910000021A120FFF71EFE0021C020FFF71AFEB4
:102920000021DA20FFF716FE00211220FFF712FE29
:1029300000218120FFF70EFE0021EF20FFF70AFEA5
:102940000021D920FFF706FE0021F120FFF702FE4B
:102950000021DB2010E00000BC01214294812142D3
:10296000C000002042820008B6860008000C01402A
:102970000008014000802142FFF7ECFD00213020DB
:10298000FFF7E8FD0021A420FFF7E4FD0021A620C9
:10299000FFF7E0FD0021AF20FFF7DCFDFFF740FE71
:1029A00008BD000008B501210820FEF719FA4FF410
:1029B0007040ADF8000010208DF8030003208DF862
:1029C000020069462A48FDF7E9FE08BD30B589B026
:1029D00005460C46FFF7E6FF0121C802FEF700FAA4
:1029E00001210420FEF7FCF94FF41060ADF820003F
:1029F00018208DF8230003208DF8220008A91D4817
:102A0000FDF7CCFEADF81850ADF814400020ADF83D
:102A10001A00ADF8160005A91748FEF719FB60204B
:102A2000ADF804000120ADF806000020ADF80A0062
:102A3000ADF80C0001A91048FEF747FB01A90E48AC
:102A4000FEF71DFC01210C48FEF76AFE08210A482A
:102A5000FEF78AFF08210848FEF7A5FF0121064876
:102A6000FEF752FF01210448FEF74EFE09B030BDCB
:102A7000000C014000080140002C014000B587B067
:102A800001210846FEF7B9F901210420FEF7A8F953
:102A90000320ADF8000004208DF80300694661486A
:102AA000FDF77CFE04A8FEF7FFFD0020ADF8100046
:102AB0004FF6FF70ADF814000020ADF81600ADF829
:102AC000120004A94FF08040FEF7C2FA00231A4614
:102AD00003214FF08040FEF7CAFE01A8FEF7F7FD84
:102AE0000A20ADF80C0001A94007FEF744FD0121C2
:102AF0008807FFF7CFF8012211469007FEF71FFE67
:102B000000214FF08040FFF793F801218807FEF77E
:102B1000FBFD07B000BD00B587B001210420FEF722
:102B20006CF901210820FEF75BF9C020ADF8000028
:102B300004208DF8030069463B48FDF72FFE04A8EA
:102B4000FEF7B2FD0020ADF810004FF6FF70ADF8B3
:102B500014000020ADF81600ADF8120004A93348A7
:102B6000FEF776FA00231A4603213048FEF77FFE6F
:102B700001A8FEF7ACFD0A20ADF80C0001A92B4816
:102B8000FEF7F9FC01212948FFF784F801221146DC
:102B90002648FEF7D4FD00212448FFF749F801211B
:102BA0002248FEF7B1FD07B000BD0146022904D05E
:102BB00003290BD0042919D10FE04FF08042928CE9
:102BC00010B200224FF080439A8411E0184A128814
:102BD00010B20022164B1A800AE0144A24321288DE
:102BE00010B20022114B24331A8001E0002000BFF4
:102BF00000BF70470D48103000880C481030008826
:102C000020F0010009491031088070474FF08040E2
:102C1000008A4FF08040008A20F001004FF0804190
:102C20000882704700080140000C01400008004085
:102C30002404004008B501210820FEF7D1F84FF424
:102C40004070ADF8000010208DF8030003208DF8CF
:102C500002006946F748FDF7A1FD08BD10B5F5482B
:102C6000001D006820F0F000F249091D08600846C8
:102C7000006840F0300008600120EF490860EF482C
:102C8000D0F8240108B9002010BD0120EA49091F2D
:102C90000860FFF734FA0020E849C1F8A401E648CB
:102CA0008038006808B10020EEE70120FFF727FA1E
:102CB0000020E149091F08600120E5E710B5DD4863
:102CC000001D006820F0F000DA49091D0860084680
:102CD000006840F0300008600020D749091F0860F4
:102CE000D649C1F8A4010120FFF709FA0120D24911
:102CF000091F0860D149C1F8A401FFF700FA10BD0F
:102D000010B50024CB48001D006820F0F000C94930
:102D1000091D08600846006840F080000860012036
:102D2000C5490860FFF7EBF90120C449C1F8A001CB
:102D3000FFF7E5F90AE0601CC4B2322C03DDFFF7AF
:102D4000BDFF002010BD0120FFF7D9F9BA48803837
:102D500000680028EFD1B849091F08600120F1E799
:102D600010B50020B449091F0860B248001D006872
:102D700020F0F000AF49091D08600846006840F0E7
:102D8000300008600020AD49C1F8A4010120FFF720
:102D9000B6F90120A849091F0860FFF7B0F9002023
:102DA000A649C1F8A00110BD10B50020A249091F15
:102DB0000860A048001D006820F0F0009D49091D32
:102DC00008600846006840F03000086001209B4918
:102DD000C1F8A401FFF793F901209749091F086082
:102DE000FFF78DF900209549C1F8A00110BD70B51D
:102DF00004469048001D006820F0F0008D49091D30
:102E000008600846006840F03000086000208A49E9
:102E1000091F0860002516E0E00987490860600680
:102E2000040E0120FFF76BF901208449C1F8A001CD
:102E3000FFF765F900208049091F08600120FFF7AE
:102E40005EF9681CC5B2082DE6DB70BD2DE9F041C6
:102E500005460E4617469846FFF700FF10B90120B9
:102E6000BDE8F0816906080EFFF7C1FFFFF748FFD4
:102E700018B9FFF723FF0120F2E73046FFF7B7FF4D
:102E8000FFF73EFF00240BE018F80400FFF7AFFF48
:102E9000FFF736FF18B9FFF711FF0020E0E7641CC9
:102EA000BC42F1DBFFF70AFF0020D9E770B5054609
:102EB00000246048001D006820F0F0005D49091DF5
:102EC00008600846006840F080000860002617E0AF
:102ED00000205949091F08600220FFF710F901205E
:102EE0005649C1F8A0016006040E534880380068B6
:102EF00008B1601CC4B20220FFF701F9701CC6B211
:102F0000082EE5DB15B1FFF72BFF01E0FFF74CFFC3
:102F1000204670BD2DE9F04106460F4614461D4679
:102F2000FFF79CFE10B90120BDE8F0817106080E84
:102F3000FFF75DFFFFF7E4FE18B9FFF7BFFE0120C2
:102F4000F2E73846FFF753FFFFF7DAFEFFF786FE9A
:102F5000012101EB4601C8B2FFF749FFFFF7D0FEA0
:102F60000DE0012C04D10020FFF7A0FF287003E042
:102F70000120FFF79BFF28706D1C601EC4B2002C5F
:102F8000EFD1FFF79BFE0020CEE770B505460E4659
:102F90000024FFF763FE2846FFF729FF641CFFF7B4
:102FA000AFFE3046FFF723FF641CFFF7A9FEFFF7D3
:102FB00055FE691CC8B2FFF71AFF641CFFF7A0FE9C
:102FC0000020FFF773FF0446FFF778FE204670BD30
:102FD0002DE9F0410746884615461E460024FFF7B6
:102FE0003DFE3846FFF703FFFFF78AFE4046FFF736
:102FF000FEFEFFF785FEFFF731FE791CC8B2FFF732
:10300000F6FEFFF77DFE00BF0DE0681EA04204D073
:103010000120FFF74BFF305503E00020FFF746FF8C
:103020003055601CC4B2AC42EFDBFFF747FE2046D0
:10303000BDE8F081000C0140A481214200802142C2
:103040002DE9F04180460D4616461F460024FFF745
:1030500005FE4046FFF7CBFEFFF752FE2846FFF77E
:10306000C6FEFFF74DFE00BF06E0385DFFF7BFFE6E
:10307000FFF746FE601CC4B2B442F6DBFFF71EFE4B
:103080000120BDE8F08170B505460E461446314674
:103090002846FFF77AFF2070012070BD37B504463F
:1030A0000D4602AB012229462046FFF7C9FF3EBD6F
:1030B0002DE9F8430746884614461D46089E6A4691
:1030C00041463846FFF7DFFF28B3601CFF2101FAB5
:1030D00000F0C4F108012944491EFF220A411043AF
:1030E00000F0FF09C5F1080006FA00F0C6B2C4F10D
:1030F000070006419DF8000000EA090000909DF8D5
:103100000000304300909DF8002041463846FFF70C
:10311000C5FFBDE8F8830020FBE7F8B506460F467B
:1031200014461D466A4639463046FFF7ACFF2DB1BE
:103130000120A0409DF80010084305E00120A040B8
:103140009DF8001021EA0000C0B200909DF8002018
:1031500039463046FFF7A2FFF8BD00001FB5012138
:103160000846FDF73DFE01210420FDF739FE4FF42E
:103170008050ADF80C0048208DF80F0003A91248CC
:10318000FDF70CFB0C210020FDF71EFC4FF48050D6
:10319000019000208DF808000C208DF80900012016
:1031A0008DF80A0001A8FDF719FA28208DF8000013
:1031B00002208DF8010001208DF802008DF8030037
:1031C0006846FDF732F91FBD00080140014600299D
:1031D00001DA484200E00846704700B503460A4657
:1031E000002B07DD0120B24908600020B149C1F879
:1031F000B00106E00020AE4908600120AD49C1F8E9
:10320000B0011846FFF7E2FFAB490880002A08DD4D
:103210000120A749083108600020A649C1F8B8017B
:1032200007E00020A249083108600120A149C1F847
:10323000B8011046FFF7CAFF9F490C39088000BD4E
:1032400070B505469D49284604F0D2FD08D39C4937
:10325000284604F0CDFE03D39A48007801280DD10A
:10326000012400209249091D08609249C1F8BC015F
:103270008F4908608F49C1F8B00100E00024204662
:1032800070BD03461846884200DD0846904200DAC9
:10329000104670472DE9FF5F044689468A4803902F
:1032A0008A48029004EB0901484204F075FD884900
:1032B00008608848006804F0A3FB0746864A874BED
:1032C00004F0AAF9054603F06DFF824908608048C2
:1032D000006804F095FB804A814BCDE9000104F0C1
:1032E0009BF905460E467B48006804F089FB0746BB
:1032F0002A46334603F088FF824603F053FF7549A0
:103300000860084601687748006804F0A5FB754925
:10331000086075497348006804F06AFE02D272487A
:103320007049086071496F48006804F061FD02D27D
:103330006E486C4908606B480299006804F08CFD87
:1033400007466448006880F000463046039904F060
:1033500083FD0546394604F087FE654908606548E7
:103360000068FFF76DFF012803D056480078012858
:1033700002D100205B4908605D48006804F0D0FC81
:1033800004B0BDE8F09F2DE9FE4F04460D465A4EAD
:103390005A4F0021204604F05CFE0290294600208E
:1033A00004F062FE01903946019804F055FD86F064
:1033B000004B00905846029904F04EFD8246009959
:1033C00004F052FE814604F0ABFC80464046BDE866
:1033D000FE8F10B5FFF7A4F80446012C07D1394839
:1033E000007808B9012000E000203649087010BDBF
:1033F00010B503F071F9424800683E490860414940
:10340000B1F9000004F0C8FC3F49086010BD2DE987
:10341000F0413E480068002847D14FF480503C49B5
:1034200008603C48007808B9012000E000203949D4
:103430000870FFF7DDFF0220FFF7B7FB4042364977
:1034400008600420FFF7B1FB40423449086031486E
:103450000078012802D10020BDE8F081FFF7B9FF14
:103460002948016823480068FFF78DFF04462B4870
:10347000016829480068FFF70DFF054667196619BE
:10348000274A51423846FFF7FCFE0746244A51427C
:103490003046FFF7F6FE064616480068FFF7D0FEF6
:1034A00018B931463846FFF798FE0020D4E70000EF
:1034B000B481214200802142402C0140000020C202
:1034C000000020421400002000002043CDCC4C3FDF
:1034D00050000020540000209A9999999999E93F49
:1034E0009999C93F5800002000401C4600401CC666
:1034F0004C0000202000002000006143713D8A3F05
:103500009C0000208800002024000020300121427F
:103510001404014048000020180000201C00002076
:103520000CE5FFFF38B5FFF75FF84BA20021084616
:10353000FFF761F949A200213C20FFF75CF949A29D
:1035400014210020FFF757F94948006800280FDAD6
:1035500048A214215020FFF74EF90C2003230090BD
:1035600043480068424214215F20FFF7FAF80DE05B
:1035700041A214215020FFF73EF90C2003230090B4
:103580003B48142102685F20FFF7EBF83BA21E21A5
:103590000020FFF730F93C48006800280FDA35A218
:1035A0001E215020FFF727F90C20032300903648F6
:1035B000006842421E215F20FFF7D3F80DE02EA2E3
:1035C0001E215020FFF717F90C20032300902E48EE
:1035D0001E2102685F20FFF7C4F82CA232210020D0
:1035E000FFF709F900212B48006804F001FC04D220
:1035F00020A232213020FFF7FEF800212548006884
:1036000004F0F6FC04D81CA232213020FFF7F3F8B6
:103610002048006804F084FB0546FFF7D7FD044608
:103620000C2003232246322100903520FFF799F821
:103630001948007820B119A232215A20FFF7DBF88F
:103640001548007820B916A232215A20FFF7D3F886
:10365000FEF7A7FF38BD0000444D50004E6F726D5D
:10366000616C0000456E636F4C45465400000000DD
:10367000180000202D0000002B000000456E636F35
:1036800052494748540000001C000020416E676CFE
:103690006500000020000020140000204F46460076
:1036A0004F4E200038B50446FB4890F82400C0B1C6
:1036B00014B10220009001E000200090F64A126848
:1036C000D17BF54A526810786B460122FFF7BEFBAA
:1036D00010B14FF0FF3038BD9DF80010EE48417436
:1036E00023E0ED48807A10B94FF0FF30F3E724B1C2
:1036F000E948407C08B10020EDE714B101200090BA
:1037000001E000200090E44A1268D17BE24A52684E
:1037100010786B460122FFF799FB10B14FF0FF3094
:10372000D9E79DF80010DC4841740020D3E738B594
:10373000002419E0D8480068C07AA04204D0D648D6
:103740000068407DA04200D10CE0D3494968087868
:103750006B4601222146FFF7DDFB10B14FF0FF3031
:1037600038BD00BF601CC4B2CB4840680079A0429D
:10377000E0DC0020F4E770B504460D46C64800685A
:10378000C07AA04204D0C4480068407DA04202D163
:103790004FF0FF3070BDC04840680079A04202DCA5
:1037A0004FF0FF30F6E7BC49496808782B46012204
:1037B0002146FFF7AFFBEDE738B50446B64890F871
:1037C0002300A04201D1002038BD14B13020009068
:1037D00001E000200090B048807C20B19DF80000FE
:1037E00040F002000090AC4890F8220020B19DF813
:1037F000000040F080000090A74A1268117DA64AA0
:10380000526810786B460122FFF720FB10B14FF091
:10381000FF30D9E7A04880F823400020D4E738B52E
:10382000044604F0700010B10120009005E014B1CE
:103830000020009001E040200090974A1268917C9F
:10384000954A526810786B460122FFF7FFFA20B1C3
:10385000002191488172481E38BD9DF8000020F07B
:1038600040018D4801730020009004F0400020B911
:103870009DF8000040F00400009004F0200020B902
:103880009DF8000040F00200009004F0100020B904
:103890009DF8000040F00100009004F0080020B9FD
:1038A0009DF8000040F0380000907B4A1268D17CFF
:1038B000794A526810786B460122FFF7C7FA20B1A7
:1038C000002175488172481EC6E724B1082C02D039
:1038D0000020FFF771FF70488472002101753220CB
:1038E000FEF731FC0020B7E738B504466A48807C13
:1038F000A04201D1002038BD002C46D0664A126893
:103900001179654A526810786B460122FFF702FB75
:1039100010B14FF0FF30EEE79DF8000020F02000DE
:1039200000905D4A126811795B4A526810786B46C4
:103930000122FFF78BFA10B14FF0FF30DBE70320D5
:10394000FEF701FC02200090534890F8220020B1BD
:103950009DF8000040F0800000904F4890F8230050
:1039600020B19DF8000040F0300000904A4A1268F3
:10397000117D494A526810786B460122FFF766FABA
:10398000002851D04FF0FF30B5E7434A1268117953
:10399000414A526810786B460122FFF7BBFA10B11A
:1039A0004FF0FF30A7E73C48807A00F0010028B1D3
:1039B0009DF8000040F02000009004E09DF8000019
:1039C00020F020000090344A12681179324A52687F
:1039D00010786B460122FFF739FA10B14FF0FF3033
:1039E00089E70320FEF7AFFB2B4890F8220010B1C7
:1039F0008020009001E000200090274890F82300EC
:103A000020B19DF8000040F030000090224A12687A
:103A1000117D214A526810786B460122FFF716FA91
:103A200010B14FF0FF3066E71B488474002062E756
:103A300008B51948807A10B94FF0FF3008BD002052
:103A40000090154A1268D17B134A526810786B4671
:103A50000122FFF7FBF910B14FF0FF30EEE70E4AFD
:103A6000126851790C4A526810786B460122FFF7B0
:103A7000EDF910B14FF0FF30E0E7074A1268117915
:103A8000054A526810786B460122FFF7DFF928B12A
:103A90004FF0FF30D2E700005C000020F74890F8BC
:103AA0002400002850D00C200090F44A12681179AC
:103AB000F24A526810786B460122FFF7C7F910B13D
:103AC0004FF0FF30BAE7C0200090EC48807A00F059
:103AD000010020B19DF8000040F020000090E74A6E
:103AE00012681179E54A526810786B460122FFF797
:103AF000ADF910B14FF0FF30A0E7E048407C10B1C5
:103B00000220009001E000200090DC4A1268D17B86
:103B1000DA4A526810786B460122FFF797F910B124
:103B20004FF0FF308AE700200090D44A12685179A4
:103B3000D24A526810786B460122FFF787F90028B5
:103B400052D04FF0FF3079E704200090CB4A126842
:103B50001179CA4A526810786B460122FFF776F94C
:103B600010B14FF0FF3069E7C448807C20B9C348EA
:103B7000807A00F0010010B94020009001E0602040
:103B80000090BE4A12681179BC4A526810786B46A0
:103B90000122FFF75BF910B14FF0FF304EE7B74855
:103BA000407C10B10120009001E000200090B34A59
:103BB0001268D17BB14A526810786B460122FFF738
:103BC00045F910B14FF0FF3038E7AC4A126851792F
:103BD000AA4A52681078A94B10330122FFF736F930
:103BE00010B14FF0FF3029E7002027E770B50446F9
:103BF000002624F00104A14890F8240008B1002018
:103C000070BD9E48807A10B94FF0FF30F8E79B48AE
:103C1000057C807A2040994908740846007CA042BF
:103C200002D04FF0FF3600E0002614B99348007D23
:103C300018B10120FFF736FD02E00020FFF732FD4A
:103C40003CB1FFF7F5FE20B18C4805744FF0FF3012
:103C5000D6E73046D4E738B504468848807A10B9AC
:103C60004FF0FF3038BDBC2C02DB0120009015E086
:103C7000622C02DB0220009010E02A2C02DB0320E1
:103C800000900BE0142C02DB0420009006E00A2CCC
:103C900002DB0520009001E0062000907748C07A02
:103CA0009DF80010884201D10020DBE7734A1268BA
:103CB0009178724A526810786B460122FFF7C6F875
:103CC00010B14FF0FF30CDE79DF800106B48C17286
:103CD0000020C7E738B50446282C02DD4FF0FF303E
:103CE00038BDDCB90020FFF767FD00208DF800002B
:103CF00007208DF80100614A1268917C5F4A526882
:103D000010786B460222FFF7A1F810B14FF0FF3098
:103D1000E6E70021594801750020E1E70120FFF79F
:103D20004BFD20208DF80000012C06D100208DF8DD
:103D300001000520FFF78FFF17E0052C06DC0120AE
:103D40008DF801000520FFF786FF0EE0142C06DC3D
:103D500002208DF801000A20FFF77DFF05E0032017
:103D60008DF801001420FFF776FF9DF80100072170
:103D700001EB8010C0B28DF80100404A1268917CBE
:103D80003E4A526810786B460222FFF75FF810B186
:103D90004FF0FF30A4E708213848817200210173F9
:103DA000012101750020FFF721FF002098E738B5B9
:103DB00004463248807A10B94FF0FF3038BD2F48A2
:103DC00090F8240010B14FF0FF30F7E72B48007D4A
:103DD00050B134B1282C04DCE0B2FFF77BFF0020A7
:103DE000ECE70020FFF776FF042C01DA042404E05E
:103DF000B4F57A7F01DD4FF47A744FF47A7090FB5A
:103E0000F4F0401EC0B200901C4A126851781B4A60
:103E1000526810786B460122FFF718F810B14FF086
:103E2000FF30CBE79DF80000401C4FF47A7191FB06
:103E3000F0F081B21148C1810146C9894810FFF7ED
:103E40000AFF0020BAE738B504460C48807A10B95A
:103E50004FF0FF3038BD022C06D0042C07D0082CC0
:103E600008D0102C0FD10BE0002000900EE00820AD
:103E700000900BE01020009008E000005C000020A3
:103E80001820009002E04FF0FF30E3E700BFF94850
:103E9000407A9DF80010B0EBE10F01D10020D9E786
:103EA000F44A1268D179F34A526810786B460122BD
:103EB000FEF7CCFF10B14FF0FF30CBE79DF80000CC
:103EC000C110EC4841720020C4E738B50446E94807
:103ED000807A10B94FF0FF3038BDFA2C09D0B4F514
:103EE000FA7F09D0B4F57A7F09D0B4F5FA6F0CD116
:103EF00008E0002000900BE00820009008E010206F
:103F0000009005E01820009002E04FF0FF30E3E75A
:103F100000BFD848007A9DF80010B0EBE10F01D146
:103F20000020D9E7D34A12689179D24A52681078B2
:103F30006B460122FEF78AFF10B14FF0FF30CBE74E
:103F40009DF80000C010CB4908720020C4E71CB5E2
:103F500080208DF80000C74A1268917CC54A5268DB
:103F600010786B460122FEF771FF10B14FF0FF3061
:103F70001CBD6420FEF7E7F800208DF80000BD4A64
:103F80001268917CBB4A526810786B460122FEF79A
:103F90005DFF10B14FF0FF30EAE7B64A1268917D3D
:103FA000B44A526810786B460622FEF7B3FF10B190
:103FB0004FF0FF30DCE79DF80500C007400F9DF88B
:103FC000031001F0010140EA41009DF8011001F0E9
:103FD000010140EA010494B1012C03D10121A5485B
:103FE000C17431E0022C03D10021A248C1742BE03E
:103FF0002146A1A002F062FC4FF0FF30B8E79D4AD5
:104000001268D1789B4A526810786B460122FEF7FD
:1040100081FF10B14FF0FF30AAE79DF8000000F0DB
:104020000F042CB99E4802F049FC4FF0FF309FE787
:10403000042C06D19BA002F041FC01218D48C174E3
:1040400002E000218B48C174FF218A488172FF2061
:1040500088490872FF2187484172C1724FF6FF718B
:10406000C181FF21017481740121017380F8221044
:10407000002180F823104175017516300160416000
:104080008160163880F8241080F82510C1844FF420
:10409000FA60FFF71AFF10B14FF0FF3068E7022017
:1040A000FFF7D1FE10B14FF0FF3061E72A20FFF794
:1040B000D2FD10B14FF0FF305AE73220FFF777FE04
:1040C00010B14FF0FF3053E70020FFF78FFD10B124
:1040D0004FF0FF304CE70020FFF706FC10B14FF027
:1040E000FF3045E70020FFF79AFB002040E77047CC
:1040F0007CB504460D465F48807A00F0700010B928
:104100004FF0FF307CBD5B4A1268117B594A526800
:1041100010786B460622FEF7FDFE10B14FF0FF301F
:10412000F0E79DF801009DF8001040EA012000B280
:1041300020809DF803009DF8021040EA012000B2A3
:1041400060809DF805009DF8041040EA012000B24F
:10415000A08015B12846FFF7CAFF0020D2E77CB542
:1041600004460D464348807A00F0080010B94FF02D
:10417000FF307CBD3F4A1268517B3E4A526810783E
:104180006B460622FEF7C6FE10B14FF0FF30F0E797
:104190009DF801009DF8001040EA012000B2208047
:1041A0009DF803009DF8021040EA012000B26080F3
:1041B0009DF805009DF8041040EA012000B2A0809F
:1041C00015B12846FFF793FF0020D2E72DE9FE4FF7
:1041D00005460C462748807A18B94FF0FF30BDE8F5
:1041E000FE8F244A1268917B224A5268107802ABF3
:1041F0000222FEF78FFE10B14FF0FF30EFE79DF87F
:1042000009009DF8081040EA012006B214B12046CA
:10421000FFF76DFF17494968C88803F0D5FD1549B8
:1042200001904968B1F9080003F0B6FD83463046B5
:1042300003F0B2FD5946009003F016FF8246019943
:1042400003F078FC81461F4903F006FC80464FF0DE
:104250008F4103F001FE074603F062FD2860002055
:10426000BDE710B588B004461CB94FF0FF3008B068
:1042700010BD29E05C000020556E737570706F7280
:1042800074656420736F6674776172652070726FF5
:1042900064756374207265762025642E0A00000020
:1042A0009099000848616C662073656E7369746943
:1042B00076697479207061727420666F756E642EF1
:1042C0000D0A000000000C42206830B9606820B977
:1042D000A06810B9002008B010BDFA4949680878F4
:1042E00006AB03221146FEF715FE10B14FF0FF306A
:1042F000F1E79DF81800082101EB201000F00F00F5
:10430000ADF800009DF8190001EB201000F00F003F
:10431000ADF802009DF81A0001EB201000F00F002C
:10432000ADF8040020684100BDF90000403091FB69
:10433000F0F000B2ADF8100060684100BDF9020075
:10434000403091FBF0F000B2ADF81200A0684100DF
:10435000BDF90400403091FBF0F000B2ADF814005C
:10436000D8494968087806AB06221146FEF7D2FD07
:1043700010B14FF0FF30AEE79DF819009DF818100E
:1043800040EA012000B2ADF808009DF81B009DF83E
:104390001A1040EA012000B2ADF80A009DF81D0095
:1043A0009DF81C1040EA012000B2ADF80C00BDF8E9
:1043B0001000BDF80810084400B2ADF81000BDF8B8
:1043C0001200BDF80A10084400B2ADF81200BDF8A2
:1043D0001400BDF80C10084400B2ADF81400BDF88C
:1043E0001000000A8DF81800BDF81000C0B28DF85A
:1043F0001900BDF81200000A8DF81A00BDF812006D
:10440000C0B28DF81B00BDF81400000A8DF81C0026
:10441000BDF81400C0B28DF81D00AA49496808789B
:1044200006AB06221146FEF711FD10B14FF0FF302A
:1044300051E700204FE70146A248007A30B1012839
:1044400007D0022809D003280FD10AE0FA200880FB
:104450000EE04FF4FA7008800AE04FF47A7008809A
:1044600006E04FF4FA60088002E00020088000BFF8
:1044700000BF0020704701469248407A30B10128C1
:1044800007D0022808D003280CD108E002200870C9
:104490000BE00420087008E00820087005E01020F8
:1044A000087002E04FF0FF30704700BF8548C07CC5
:1044B00018B108784006000E08700020F4E70146A5
:1044C0008048C07A082817D2DFE800F01704070AEE
:1044D0000D101318BC20088013E06220088010E043
:1044E0002A2008800DE0142008800AE00A200880B5
:1044F00007E00520088004E000BF00BF002008801E
:1045000000BF00BF0020704701466E4890F82400AD
:1045100010B14FF0FF3070476A48C0890880002012
:10452000F9E7014600200880401E704701464FF021
:10453000FF30704701466348007A30B1012807D048
:10454000022808D003280CD108E05F4808600BE07F
:104550005E48086008E05E48086005E05D48086065
:1045600002E04FF0FF30704700BF0020FBE701463C
:104570005448407A30B1012808D002280AD00328D4
:1045800010D10BE04FF4804008800EE041F69C70A3
:1045900008800AE04FF48050088006E04FF4006085
:1045A000088002E04FF0FF30704700BF4548C07CF4
:1045B00010B10888401008800020F5E70146414806
:1045C000007C08700020704701463E48807A10B198
:1045D0000120087001E0002008700020704738B505
:1045E00004463848807A10B94FF0FF3038BD354A5C
:1045F0001268117C334A526810786B460222FEF72B
:1046000089FC10B14FF0FF30F0E79DF801009DF8F4
:10461000001040EA012000B220800020E6E72DE9EA
:10462000FE4F0746884692461D46DDF830B000260C
:104630000024244890F8240010B1601EBDE8FE8FCD
:10464000002028701F48807A10B94FF0FF30F5E73E
:104650001C48007C10B94FF0FF30EFE71948007C90
:1046600000F0400008B1B01CC6B21648007C00F053
:10467000200008B1B01CC6B21248007C00F0100047
:1046800008B1B01CC6B20F48007C00F0080008B1A9
:10469000B01DC6B20B4A1268917A0A4A5268107865
:1046A0006B460222FEF736FC10B14FF0FF30C5E733
:1046B0009DF801009DF8001040EA0129B1450BDA90
:1046C0000020BBE75C0000200000034300008342A1
:1046D0003333034233338341FC4840684088B9EBAD
:1046E000600F17DDF94A1268517CF84A5268107859
:1046F0006B460122FEF70EFC10B14FF0FF309DE734
:104700009DF8000000F0100020B1FFF791F96FF064
:10471000010093E75046FFF7EAFCEC4A1268D17AB1
:10472000EA4A526810786B463246FEF7F3FB10B146
:104730004FF0FF3082E799FBF6F0401E8BF8000047
:1047400000202870B4422AD0E048007C00F0080025
:1047500028B3601C1DF800001DF8041040EA012079
:1047600000B2A8F80000E01C1DF80010A01C1DF805
:10477000000041EA002000B2A8F80200601D1DF808
:104780000010201D1DF8000041EA002000B2A8F82A
:104790000400287840F008002870A01D84B2B442BC
:1047A00013D0CA48007C00F0400070B1601C1DF8B6
:1047B00000001DF8041040EA012000B2388028787B
:1047C00040F040002870A01C84B2B44213D0BF480F
:1047D000007C00F0200070B1601C1DF800001DF886
:1047E000041040EA012000B27880287840F02000D0
:1047F0002870A01C84B2B44213D0B448007C00F0EE
:10480000100070B1601C1DF800001DF8041040EA93
:10481000012000B2B880287840F010002870A01C59
:1048200084B200200AE7F8B504460F461646A748AA
:1048300090F8240010B94FF0FF30F8BDA348807AFB
:1048400010B94FF0FF30F8E7A04A1268917A9F4AFA
:10485000526810786B460222FEF75CFB10B14FF0F5
:10486000FF30EAE79DF801009DF8001040EA0125BD
:10487000A54203DA00203070401EDEE7934840680E
:104880004088B5EB600F17DD904A1268517C8F4A63
:10489000526810786B460122FEF73CFB10B14FF0D6
:1048A000FF30CAE79DF8000000F0100020B1FFF7CC
:1048B000BFF86FF00100C0E7E2B2844B1B68D97A01
:1048C000824B5B6818783B46FEF724FB10B14FF033
:1048D000FF30B2E795FBF4F0401E30700020ACE7EB
:1048E00001467A4880F82210002070477CB50546C2
:1048F00076494968087801AB04220D21FEF70AFBCE
:1049000008B107207CBD9DF80700C0F301109DF899
:10491000041001F0E00140EAE1008DF800009DF88C
:104920000700C0F381009DF8051001F0E00140EAA6
:10493000E1008DF801009DF8070000F003009DF8EC
:10494000061001F0E00140EAE1008DF802000024C9
:104950001CE01DF8040018B9002045F8240013E0FD
:104960005B4845F8240006E055F82400594903F057
:1049700073FA45F824001DF80400401EC0B20DF87B
:1049800004000028F0D100BF601CC4B2032CE0DB9F
:104990000020B7E72DE9FE4F06460F460025684682
:1049A000FFF7A4FF002442E056F8240057F8241033
:1049B000A0EB010ABAF1000F01DB514601E0CAF198
:1049C0000001084603F0E8F983464FF08F4103F0F9
:1049D000B1F880465DF82400002103F06DF916D08F
:1049E0005DF82410404603F0A5F882464FF07E5152
:1049F00003F03AFB814629F0004A3748416A5046A5
:104A000003F0F6FA12D20120A04005430EE032482E
:104A1000C169404603F0ECF905D32F48016A4046CE
:104A200003F0E6FA02D20120A0400543641C032CE7
:104A3000BADB2846BDE8FE8F2DE9FC5F06460F462F
:104A4000002522494968087801AB03220D21FEF7B1
:104A500061FA10B10720BDE8FC9F9DF8040000F04A
:104A60001F008DF804009DF8050000F01F008DF870
:104A700005009DF8060000F01F008DF806000024D8
:104A800062E056F8240057F82410A0EB010BBBF1AC
:104A9000000F01DB594601E0CBF10001084603F0AD
:104AA0007BF94FF08F41009003F044F8814601A854
:104AB000005DC0B30849086803F086F9834659468B
:104AC000064803F037F880460FE000005C00002045
:104AD0007B14AE3E1D5A843FD08C000800B04C457C
:104AE000FE49404603F0B8F9804601A8005D401E2B
:104AF000C0B201A908550028F2D14146484603F04A
:104B000019F883464FF07E5103F0AEFA82462AF040
:104B1000004BF3488169584603F06AFA13D201202A
:104B2000A04005430FE0FFE7ED480169484603F068
:104B30005FF905D3EA484169484603F059FA02D2C1
:104B40000120A0400543641C032C9ADB284682E721
:104B50002DE9F04F87B005460C46914601208DF8AF
:104B6000100000208DF81100DE4A1268917CDD4AA9
:104B70005268107804AB0222FEF768F920B14FF0BA
:104B8000FF3007B0BDE8F08FC820FDF7DCFA002049
:104B90008DF81000D34A1268D17BD24A526810783F
:104BA00004AB0122FEF752F910B14FF0FF30E8E7F5
:104BB000CC4A12685179CB4A5268107804AB012272
:104BC000FEF744F910B14FF0FF30DAE7C54A12683A
:104BD000917CC44A5268107804AB0122FEF736F982
:104BE00010B14FF0FF30CCE7BE4A1268D17DBD4A0C
:104BF0005268107804AB0122FEF728F910B14FF08B
:104C0000FF30BEE7B74A12681179B64A5268107889
:104C100004AB0122FEF71AF910B14FF0FF30B0E7F4
:104C20000C208DF81000AF4A12681179AD4A526815
:104C3000107804AB0122FEF709F910B14FF0FF30F4
:104C40009FE70F20FDF77FFAA648806A407A8DF82B
:104C50001000A44A12689178A24A5268107804ABF6
:104C60000122FEF7F3F810B14FF0FF3089E79D48BD
:104C7000806A007A8DF810009A4A12685178994A31
:104C80005268107804AB0122FEF7E0F810B14FF043
:104C9000FF3076E7B9F1000F07D09248806A807A3A
:104CA00040F0E0008DF8100004E08E48806A807AC1
:104CB0008DF810008B4A126891798A4A52681078F0
:104CC00004AB0122FEF7C2F810B14FF0FF3058E7F5
:104CD000B9F1000F07D08348806AC07A40F0E00045
:104CE0008DF8100003E07E48C07A8DF810007D4AF0
:104CF0001268D1797B4A5268107804AB0122FEF722
:104D0000A5F810B14FF0FF303BE7B9F1000F02D02A
:104D1000C820FDF718FA40208DF81000714A12687B
:104D20001179704A5268107804AB0122FEF78EF8B0
:104D300010B14FF0FF3024E778208DF81000694A59
:104D400012685179674A5268107804AB0122FEF765
:104D50007DF810B14FF0FF3013E761498889FDF706
:104D6000F2F900208DF810005E4A126851795D4A10
:104D70005268107804AB0122FEF768F810B14FF0CA
:104D8000FF30FEE6574A1268917A564A5268107808
:104D900004AB0222FEF7BEF810B14FF0FF30F0E690
:104DA0009DF811009DF8101040EA012B0C209BFB90
:104DB000F0F0C6B20020A86068602860A060606063
:104DC0002060824665E0474A1268D17A454A5268B7
:104DD000107804AB0C22FEF79DF810B14FF0FF30B5
:104DE000CFE69DF811009DF8101040EA012000B2B6
:104DF000ADF808009DF813009DF8121040EA01205C
:104E000000B2ADF80A009DF815009DF8141040EAB4
:104E1000012000B2ADF80C00BDF90810206808446C
:104E20002060BDF90A10606808446060BDF90C108C
:104E3000A0680844A0609DF817009DF8161040EA8D
:104E4000012000B2ADF800009DF819009DF818107F
:104E500040EA012000B2ADF802009DF81B009DF869
:104E60001A1040EA012000B2ADF80400BDF90010AC
:104E7000286808442860BDF9021068680844686022
:104E8000BDF90410A8680844A8600AF1010000F008
:104E9000FF0AB24597DB1248D0F800C02868C11756
:104EA000090441EA1041070462460023384601F034
:104EB000E0FC32460023CDE9020101F0DAFC286073
:104EC0000748D0F800C06868C117090441EA1041DA
:104ED000070462460023384606E0000054E3853F9D
:104EE000D08C00085C00002001F0C3FC3246002397
:104EF000CDE9020101F0BDFC6860FE48D0F800C0B9
:104F0000A868C117090441EA10410704624600235A
:104F1000384601F0AEFC32460023CDE9020101F033
:104F2000A8FCA860F348D0F804C02168C8170004A2
:104F300040EA11480F04624600233846414601F01A
:104F400098FC32460023CDE9020101F092FC20607A
:104F5000E848D0F804C06068C117090441EA10416C
:104F6000070462460023384601F083FC32460023E2
:104F7000CDE9020101F07DFC6060DE48D0F804C09C
:104F8000A068C117090441EA1041070462460023E2
:104F9000384601F06EFC32460023CDE9020101F0F3
:104FA00068FCA060A068002804DDA068A0F580303F
:104FB000A06003E0A06800F58030A0600020E0E57C
:104FC00038B50446CC4890F82400A04201D1002016
:104FD00038BD24B3C84890F8250010B94FF0FF3011
:104FE000F6E70020FEF75EFB0020FEF77DFCC249DD
:104FF000C88CFEF7DCFE00200090BF4949680878A5
:105000006B4601222321FDF721FF0121BA4880F8D8
:1050100024100120FEF746FBFEF70AFD13E00020F6
:10502000FEF740FBB448007C0090B349496808781B
:105030006B4601222321FDF709FF0021AE4880F8CD
:105040002410FEF7F5FC0020C2E72DE9F04F8DB0EB
:1050500083460F4602200C90A74890F8240020B108
:105060000020FFF7ADFF012600E0002603A8FFF7B0
:10507000E2F905A8FFF7FFF901A8FFF720FA02A857
:10508000FFF742FA9C4890F80AA004A8FFF796FAA6
:10509000002407E0002239465846FFF759FD00B9C1
:1050A00002E0641C022CF5DB00BF022C01D10025BC
:1050B00028E0002407E0012206A909A8FFF748FD1F
:1050C00000B902E0641C022CF5DB00BF022C01D108
:1050D000002517E006A93846FFF75CFC00F0FF0842
:1050E00009A95846FFF7A8FC00F0FF090025B9F10F
:1050F000000F01D145F00105B8F1000F01D145F0D5
:10510000020500BFFF207C490872FF217A484172E6
:10511000C1724FF6FF71C181FF21817201740121BB
:105120000173BDF80C00FEF7D0FE9DF81400FEF7E9
:105130008AFEBDF80400FEF78EFDBDF80800FEF7FC
:1051400036FE5046FEF76BFB9DF81000FEF74EFD55
:1051500016B10120FFF734FF28460DB0BDE8F08FEF
:10516000F8B504460D46164616B94FF0FF30F8BDA7
:105170006148807A10B94FF0FF30F8E720128DF8BF
:105180000000E0B28DF801009DF8010028445A4962
:1051900049684989884202DD4FF0FF30E7E7564A07
:1051A0001268117E544A526810786B460222FDF74D
:1051B0004DFE10B14FF0FF30D9E7EAB24E4B1B68FD
:1051C000597D4D4B5B6818783346FDF73FFE10B1B3
:1051D0004FF0FF30CBE70020C9E7F8B504460D4695
:1051E000164616B94FF0FF30F8BD4348807A10B923
:1051F0004FF0FF30F8E720128DF80000E0B28DF894
:1052000001009DF8010028443B49496849898842CA
:1052100002DD4FF0FF30E7E7374A1268117E364A69
:10522000526810786B460222FDF710FE10B14FF065
:10523000FF30D9E7EAB2304B1B68597D2E4B5B68D3
:1052400018783346FDF766FE10B14FF0FF30CBE71C
:105250000020C9E72DE9F04385B005460E4690468B
:105260009946254890F8250020B14FF0FF3005B051
:10527000BDE8F08316B94FF0FF30F8E7002423E0D3
:10528000281B102801DD102000E0281B87B23219EE
:1052900039462046FFF764FF10B14FF0FF30E6E7D4
:1052A00001AA39462046FFF798FF10B14FF0FF30B2
:1052B000DDE730193A4601A901F07CFB10B16FF02F
:1052C0000100D4E7E01984B2AC42D9DB4FEA2820D0
:1052D0008DF8000008F0FF008DF80100064A126802
:1052E000917E054A526810786B460222FDF7AEFDAA
:1052F00038B103E0D08C00085C0000204FF0FF3094
:10530000B5E701218A4880F82510A0F826900020F2
:10531000ADE70146864890F82400087000207047E9
:1053200002464FF0FF30704701464FF0FF307047A4
:10533000F8B505460F461446002C70D0B5F5FF5F52
:1053400001DDFF2605E0202D01DA012601E0C5F38D
:10535000471607B90127282C02DD4FF0FF30F8BDB2
:105360007348407D28BB724890F8240038B1002073
:10537000FFF726FE01216E4880F8201003E000218F
:105380006B4880F820106A481630FFF754F86848D8
:105390001830FFF770F866481A30FFF790F8644845
:1053A0001C30FFF7B1F86248817A81771F30FFF730
:1053B00005F90020FEF776F90020FEF78BFC0020AF
:1053C0008DF800005A4A12689178594A526810784C
:1053D0006B460122FDF73AFD10B14FF0FF30BEE7FA
:1053E00040208DF80000524A1268D17B504A526822
:1053F00010786B460122FDF729FD00B165E08DF8BC
:1054000000608DF801704A4A1268117A484A526861
:1054100010786B460222FDF719FD08B155E047E010
:105420000520FCF790FE4248407A072101EBC000BE
:10543000C0B28DF800003E4A1268D1793C4A5268E9
:1054400010786B460122FDF701FD00B13DE0202000
:105450008DF80000012C03D100208DF801000EE032
:10546000052C03DC01208DF8010008E0142C03DC7E
:1054700002208DF8010002E003208DF801009DF864
:105480000100072101EB8010C0B28DF80100284A0D
:105490001268917C264A526810786B460222FDF70A
:1054A000D5FC00B111E0012121484175002056E7EB
:1054B0001F4A1632002103E0505C00B105E0491C90
:1054C0000C29F9D34FF0FF3049E7FF201849087243
:1054D000FF2117484172C1724FF6FF71C181FF2150
:1054E00081720174012101730146887FFEF797F9EB
:1054F0000F49C88AFEF7E9FC0D49087EFEF7A3FCB8
:105500000B49488BFEF7A7FB0949888BFEF74FFC38
:105510000749C87FFEF76AFB054890F8200010B1E4
:105520000120FFF74DFD002101484175002016E7DD
:105530005C00002010B5C8234FF48062F74940F6A4
:10554000F630FFF787FE10BD10B586B00446F4A014
:1055500000680390F3A000680290F3A00068019037
:10556000F2A00068009004F0030003A9085C8DF825
:10557000140003A8C4F3C101405C8DF8150003A812
:10558000C4F38111405C8DF8160004F0030002A9F9
:10559000085C8DF8100002A8C4F3C101405C8DF8CE
:1055A000110002A8C4F38111405C8DF8120005AA15
:1055B000032140F22640FFF7D3FD18B14FF0FF3032
:1055C00006B010BD04AA032140F22A40FFF7C8FD2F
:1055D00010B14FF0FF30F3E7019805900098049068
:1055E00004F0040058B19DF8140040F001008DF85B
:1055F00014009DF8100040F001008DF8100004F038
:10560000200058B19DF8150040F001008DF81500FC
:105610009DF8110040F001008DF8110004F4807035
:1056200058B19DF8160040F001008DF816009DF865
:10563000120040F001008DF8120005AA03214FF47A
:105640008860FFF78DFD10B14FF0FF30B8E704AA76
:10565000032140F23140FFF783FD10B14FF0FF30DE
:10566000AEE7B34804810020AAE71FB50446B0485E
:10567000007A00F0030054F820000190AC48007A52
:1056800000F0040010B1019840420190A848007A4F
:10569000C0F3C10054F820000290A548007A00F041
:1056A000200010B1029840420290A148007AC0F355
:1056B000811054F8200003909D48008900F4807008
:1056C00010B10398404203909A49019880FB010170
:1056D000800F40EA810001909649029880FB0110FA
:1056E000820042EA917002909249039880FB011077
:1056F000820042EA917003900198000E8DF800003C
:105700000198000C8DF801000198000A8DF8020044
:105710000198C0B28DF803006A4604214FF47470FA
:10572000FFF71EFD18B14FF0FF3004B010BD029816
:10573000000E8DF800000298000C8DF80100029810
:10574000000A8DF802000298C0B28DF803006A4684
:1057500004214FF47570FFF703FD10B14FF0FF30D7
:10576000E3E70398000E8DF800000398000C8DF815
:1057700001000398000A8DF802000398C0B28DF86A
:1057800003006A4604214FF47670FFF7E9FCCCE78A
:1057900070B588B0064601A8FEF7E9FEBDF8040022
:1057A0000021C90341EA5045C4036148007A00F072
:1057B000030056F8200005905D48007A00F00400D0
:1057C00010B10598404205905948007AC0F3C100D5
:1057D00056F8200006905648007A00F0200010B1DC
:1057E0000698404206905248007AC0F3811056F85D
:1057F000200007904E48008900F4807010B107988F
:10580000404207900598C117A0FB042301FB043117
:1058100000FB0510810041EA927005900698C117BF
:10582000A0FB042301FB043100FB0510810041EAC9
:10583000927006900798C117A0FB042301FB043166
:1058400000FB0510810041EA927007900598000E58
:105850008DF808000598000C8DF809000598000ADD
:105860008DF80A000598C0B28DF80B000698000E5E
:105870008DF80C000698000C8DF80D000698000AB3
:105880008DF80E000698C0B28DF80F000798000E34
:105890008DF810000798000C8DF811000798000A89
:1058A0008DF812000798C0B28DF8130002AA0C21DF
:1058B0004FF42570FFF754FC08B070BD30B585B0CB
:1058C00004461DA207CA02AB07C3C82C03DD4FF074
:1058D000FF3005B030BDC82090FBF4F0401E85B20B
:1058E000280A8DF80000E8B28DF801006A4602210E
:1058F00040F21620FFF734FC10B14FF0FF30E8E71C
:1059000002AA0C2140F6C120FFF72AFC10B14FF08B
:10591000FF30DEE7064884810020DAE7F88C0008D3
:105920004CCD6C000CC92C0036567600264666001D
:10593000C004002009E3CA02FEF2ABC4AAF1DFDF13
:10594000BBAFDFDF0146FC4880890880002070473C
:105950002DE9FC4706460F4606F0070010B1B7F5E3
:10596000C86F03DD4FF0FF30BDE8FC87384602F01A
:105970002BFA8146F14902F0DDF880466846FEF7D1
:105980007AFD9DF80000022806D0042816D00828C9
:1059900026D0102848D135E04FF08D41404602F026
:1059A0005BFA814602F0D8F984B2E549404602F03C
:1059B00053FA814602F0D0F985B238E04FF08C41BD
:1059C000404602F049FA814602F0C6F984B2DD4948
:1059D000404602F041FA814602F0BEF985B226E067
:1059E0004FF08B41404602F037FA814602F0B4F99D
:1059F00084B2D549404602F02FFA814602F0ACF954
:105A000085B214E04FF08A41404602F025FA814603
:105A100002F0A2F984B2CD49404602F01DFA814657
:105A200002F09AF985B202E04FF0FF309CE700BF28
:105A300020128DF80400E0B28DF8050028128DF8D0
:105A40000600E8B28DF8070006F00100A0B101AA37
:105A500002214FF4EA70FFF783FB10B14FF0FF30E3
:105A600082E70DF1060202214FF49270FFF778FBF6
:105A700010B14FF0FF3077E706F00200A0B101AAA5
:105A800002214FF4EC70FFF76BFB10B14FF0FF30C9
:105A90006AE70DF1060202214FF49470FFF760FBF4
:105AA00010B14FF0FF305FE706F00400A0B101AA8B
:105AB00002214FF4EE70FFF753FB10B14FF0FF30AF
:105AC00052E70DF1060202214FF49670FFF748FBF2
:105AD00010B14FF0FF3047E7002045E738B50446E6
:105AE0000020009004F0010020B19DF8000040F07B
:105AF0003000009004F0020020B19DF8000040F05A
:105B00000C00009004F0040020B19DF8000040F06B
:105B1000030000906A4601214FF4A470FFF720FBB8
:105B200038BD38B50446012C01DA012402E0042C0A
:105B300000DD0424601EC0B200906A46012140F2DC
:105B40004F10FFF70DFB38BD38B50446052094FB18
:105B5000F0F085B228128DF80000E8B28DF801004F
:105B60006A4602214FF4EF70FFF7FAFA38BD38B5F4
:105B70000446052094FBF0F085B228128DF8000051
:105B8000E8B28DF801006A4602214FF4ED70FFF78C
:105B9000E7FA38BDF8B505460E464FF47A7095FB26
:105BA000F0F000FB06F4200E8DF80000200C8DF8BC
:105BB0000100200A8DF80200E0B28DF803006A4669
:105BC00004214FF4AE70FFF7CBFAF8BD38B50446A8
:105BD000052094FBF0F084B220128DF80000E0B2B2
:105BE0008DF801006A4602214FF4AD70FFF7B8FA54
:105BF00038BD38B50446052094FBF0F084B220127D
:105C00008DF80000E0B28DF801006A4602214FF4E1
:105C1000AC70FFF7A5FA38BD38B5044614B94FF09B
:105C2000FF3038BD6A4604214FF45870FFF7D5FAAB
:105C300010B14FF0FF30F4E79DF8000000069DF82A
:105C4000011040EA01409DF8021040EA01209DF851
:105C50000310084320600020E3E738B50446200E17
:105C60008DF80000200C8DF80100200A8DF802004C
:105C7000E0B28DF803006A4604214FF45870FFF734
:105C80006FFA38BD38B5044614B94FF0FF3038BD4F
:105C90006A4604214FF47170FFF79FFA10B14FF07C
:105CA000FF30F4E79DF8000000069DF8011040EA7F
:105CB00001409DF8021040EA01209DF803100843BE
:105CC00000EB8000800020600020E0E738B504464B
:105CD0001420B4FBF0F4200E8DF80000200C8DF899
:105CE0000100200A8DF80200E0B28DF803006A4638
:105CF00004214FF47170FFF733FA38BD38B504460C
:105D000064B120208DF8000028208DF8010030209B
:105D10008DF8020038208DF8030004E0A32204214E
:105D2000684600F073FE6A46042140F69E20FFF7A5
:105D300017FAFDF77DFE38BDC0040020000048437F
:105D4000000040460000C045000040450000C0443F
:105D500038B5044664B1C0208DF80000C2208DF82B
:105D60000100C4208DF80200C6208DF8030004E075
:105D70008B220421684600F049FE6A46042140F661
:105D80009820FFF7EDF9FDF753FE38BD3EB5044608
:105D90006CB1FDA1D1E900208968CDE90020029114
:105DA0006A4609214FF49760FFF7DAF93EBDF9A280
:105DB000D2E900109268CDE9010200916A460921FA
:105DC0004FF49760FFF7CCF9F0E73EB504460220A8
:105DD0008DF80000CA208DF80100E3208DF8020044
:105DE00009208DF803006A4604216820FFF7B8F9FE
:105DF000A3208DF8000004F0400048B1C0208DF8C9
:105E00000100C8208DF80200C2208DF8030006E0D2
:105E1000A3208DF801008DF802008DF8030004F432
:105E2000C07048B1C4208DF80400CC208DF8050066
:105E3000C6208DF8060006E0A3208DF804008DF83A
:105E400005008DF80600A3208DF807008DF80800E6
:105E50008DF809006A460A2140F6A720FFF780F96D
:105E600004F0030018B120208DF8000002E0D820D3
:105E70008DF800006A46012140F6B620FFF770F960
:105E800004F0200018B10120FFF780FF02E000209D
:105E9000FFF77CFF04F4C07008B304F4807060B1B5
:105EA000B2208DF800008B208DF80100B6208DF80F
:105EB00002009B208DF803000BE0B0208DF800005D
:105EC00080208DF80100B4208DF8020090208DF81C
:105ED00003006A46042140F6A220FFF741F904F0CE
:105EE000010020B3F8208DF800006A4601214FF42C
:105EF0000B60FFF735F9FA210720FFF729FD07208E
:105F0000FFF7ECFD0120FFF70CFE6420FFF71CFEFD
:105F10004FF4FA70FFF72BFEC821A148FFF73AFEB5
:105F20002820FFF753FE0A20FFF763FE08E0D82081
:105F30008DF800006A4601214FF40B60FFF710F95D
:105F400004F0020018B1D9208DF8000002E0D8203A
:105F50008DF800006A46012140F23D70FFF700F91C
:105F600004F0040018B10120FFF7F2FE02E0002067
:105F7000FFF7EEFE04F0100018B10120FFF7BEFE9F
:105F800002E00020FFF7BAFE44F00800854948818E
:105F9000FDF74EFD00208349887304F0400018B1DE
:105FA0000846807B801D887304F4C07020B17D4852
:105FB000807B801D7B49887304F0140020B17948F0
:105FC000807B10307749887304F0030020B1754856
:105FD000807B001D7349887300203EBD01467148D7
:105FE00040890880002070472DE9F0410446E078A0
:105FF00000F0C006E07800F03F05607800F0010096
:1060000098B1EF102846E91705EB5171C910A5EBBF
:10601000C101491C01F0FF086248006820B16148D5
:10602000414602683846904700BF607800F008009B
:1060300030B15C48406818B1B0115A4A516888477D
:106040000020BDE8F08110B586B0044656A207CA0C
:1060500003AB07C357A207CA8DE80700012C09D07C
:10606000022C0ED103AA0B2140F68220FFF778F80C
:1060700006B010BD6A460B2140F68220FFF770F88B
:10608000F6E74FF0FF30F3E72DE9F04F8DB007460C
:10609000884615469946DDE9166B002400203080BD
:1060A0004049887B5A4605A9FEF7BDFB18B1601E22
:1060B0000DB0BDE8F08F3B48807A00F01400002856
:1060C00061D09DF8140000069DF8151040EA0140CB
:1060D0009DF8161040EA01209DF81710084328602B
:1060E0009DF8180000069DF8191040EA01409DF83F
:1060F0001A1040EA01209DF81B10084368609DF8C3
:106100001C0000069DF81D1040EA01409DF81E107D
:1061100040EA01209DF81F100843A8609DF8200068
:1061200000069DF8211040EA01409DF8221040EA47
:1061300001209DF823100843E86004F11000C4B268
:10614000286800140190686800140290A868001480
:106150000390E8680014049001984043029901FB01
:106160000100039901FB0100049901FB010ABAF146
:10617000706F02DBBAF1885F22DDFDF759FC002069
:106180003080401E94E721E0B8AAB38DB4980D3555
:106190005D000000B8AAAAAAB088C3C5C700000065
:1061A00009E3CA02C0040020D8B1B9F38BA391B6A9
:1061B00009B4D900DAB1B9F38BA391B6DAB4DA0035
:1061C000B6F9000040F48070308000BF3448807A17
:1061D00000F0400020B305A9601C085C095D40EA9E
:1061E000012000B2A8F8000005A9E01C095C05AA7E
:1061F000A01C105C41EA002000B2A8F8020005A92A
:10620000601D095C201D105C41EA002000B2A8F866
:106210000400A01DC4B2B6F9000040F008003080B0
:106220001F48408900F4C07008B305A9601C085CD1
:10623000095D40EA012000B2388005A9E01C095C34
:1062400005AAA01C105C41EA002000B2788005A9D4
:10625000601D095C201D105C41EA002000B2B8807E
:10626000A01DC4B2B6F9000040F0700030800C48A8
:10627000807A00F0030018B105A90819FFF7B4FEF1
:106280004846FDF734FF002012E70146044801604C
:10629000002070470146024841600020704700001E
:1062A000C0040020014691F90020002A01DD0020F1
:1062B0001EE091F90020002A01DA042018E091F98B
:1062C0000120002A01DD012012E091F90120002ABD
:1062D00001DA05200CE091F90220002A01DD0220FC
:1062E00006E091F90220002A01DA062000E00720EA
:1062F000704770B505462846FFF7D4FF0446E81CF2
:10630000FFF7D0FF44EAC00084B2A81DFFF7CAFF20
:1063100044EA801084B2204670BD70B588B002A9EE
:1063200005A8FEF792FE0446072C3FD101A8FEF710
:1063300001F9059801F030FD0646019901F08CFD48
:10634000054601F0EDFC0590069801F025FD064696
:10635000019901F081FD054601F0E2FC06900798E5
:1063600001F01AFD0646019901F076FD054601F09F
:10637000D7FC079005A8FFF778F96846FEF7F7F80D
:10638000BDF80010029848430290BDF80010039831
:1063900048430390BDF8001004984843049002A8B5
:1063A000FFF7F6F9FEA000F089FA00BF08B070BD53
:1063B0002DE9F04304460D46DDE907670021012081
:1063C00041E0DFF800C43CF81080A0F1010CDFF8D8
:1063D000F49329F81C8009F1160C3CF81090A0F1F8
:1063E000010CDFF8E08308F1160828F81C9008F18A
:1063F000160C3CF81090A0F1010C08F1160828F8D2
:106400001C9008F1160C3CF81090A0F1010C08F15A
:10641000160828F81C9008F1160C3CF81090A0F112
:10642000010C08F1160828F81C9008F1160C3CF82D
:106430001090A0F1010C08F1160828F81C9000F14A
:10644000010C0CF0FF000A28BBDBDFF878C3ACF8C6
:106450001240ACF82850ACF83E20ACF85430ACF800
:106460006A60ACF880700021002008E0DFF854C3B7
:106470003CF910C0614400F1010C0CF0FF000A2847
:10648000F4DB4FF00A0C91FBFCFC0FFA8CFCDFF8FC
:106490003483A8F814C0002100200AE0DFF824C3E8
:1064A0000CF1160C3CF910C0614400F1010C0CF029
:1064B000FF000A28F2DB4FF00A0C91FBFCFC0FFAFC
:1064C0008CF8DFF800C3ACF82A80002100200AE035
:1064D000DFF8F0C20CF12C0C3CF910C0614400F163
:1064E000010C0CF0FF000A28F2DB4FF00A0C91FBC4
:1064F000FCFC0FFA8CF8DFF8CCC2ACF8408000212D
:1065000000200AE0DFF8BCC20CF1420C3CF910C0DC
:10651000614400F1010C0CF0FF000A28F2DB4FF09F
:106520000A0C91FBFCFC0FFA8CF8DFF898C2ACF86F
:106530005680002100200AE0DFF888C20CF1580CD8
:106540003CF910C0614400F1010C0CF0FF000A2876
:10655000F2DB4FF00A0C91FBFCFC0FFA8CF8DFF831
:1065600064C2ACF86C80002100200AE0DFF854C25D
:106570000CF16E0C3CF910C0614400F1010C0CF000
:10658000FF000A28F2DB4FF00A0C91FBFCFC0FFA2B
:106590008CF8DFF830C2ACF88280BDE8F08338B503
:1065A0000446032302226B21D0200094FCF780FDD7
:1065B00038BD38B50446022304221B21D0200094A4
:1065C000FCF776FD38BD38B50446022304221C21B1
:1065D000D0200094FCF76CFD38BD10B5044623466E
:1065E00006226B21D020FCF798FD10BD10B5764B2C
:1065F00001227521D020FCF7EBFC7348007810BD18
:1066000010B5FFF7F3FF682801D1012010BD00206D
:10661000FCE710B50446234605226A21D020FCF78A
:106620007CFD10BD10B50446234601223721D02041
:10663000FCF773FD10BD10B50220FFF7B0FF03207B
:10664000FFF7B7FF0020FFF7BEFF0020FFF7C5FFF1
:106650000020FFF7DEFF0020FFF7E4FF10BD38B594
:10666000002000906B46012275216820FCF752FC47
:106670009DF8000068280ED000BF5448006800F460
:10668000E06053490843001D50490860BFF34F8F35
:1066900000BF00BFFEE7FDF75AFCE0B97820FDF728
:1066A000BEF87820FDF7A2FAC820FDF780FBFEF7C0
:1066B00041FF4848FFF71DFE0446FEF745FF40F244
:1066C0007310FFF782FBC820FFF7F8F8FFF725FEED
:1066D0000120FEF775FC38BD2DE9F04F8DB00AA8FA
:1066E0003D490BAB06AACDE900103C493C48FFF7F9
:1066F000CBFC3948008800F4807000287AD00698D6
:1067000001F04AFB04464FF09D4101F013FA354970
:106710000860079801F040FB04464FF09D4101F0EE
:1067200009FA31490860089801F036FB04464FF039
:106730009D4101F0FFF92D490860099801F02CFBFB
:1067400004464FF09D4101F0F5F9294908602748BA
:1067500001684FF0804001F07FFB01902348016801
:10676000019801F079FB82461F4801684FF04040D4
:1067700001F072FB01901C480168019801F06CFB6C
:106780008346514601F070FC81464FF07E5101F086
:1067900063F9044601F034F9CDE9020111482AE019
:1067A00073657474696E67206269617320737563C1
:1067B00063657366756C6C79202E2E2E2E2E2E0D31
:1067C0000A000000DE040020D00400200CED00E0F0
:1067D0000000FA05B0000020940000208E00002088
:1067E00088000020A0000020A4000020A8000020B5
:1067F000AC0000202FE001684FF0804001F02CFB3E
:10680000834616480168584601F026FB8146144825
:1068100001684FF0804001F01FFB8346114801687A
:10682000584601F019FB8246494601F015F9044625
:1068300001F0E6F80746DDE9022300F0F3FB4FF034
:106840006632094BCDE9040100F0E6FE054600F092
:10685000A9FC064908600DB0BDE8F08FA400002037
:10686000A8000020AC00002066A64C409C00002040
:10687000704710B54C1084EA530404D54042C1F16E
:10688000000138BF491E1B4204D55242C3F1000328
:1068900038BF5B1E00F0C6F814F0804F04D04042B1
:1068A000C1F1000138BF491E14F0004F04D052421C
:1068B000C3F1000338BF5B1E10BD00000FB40449D4
:1068C00010B503AA029800F07DF910BC5DF814FB26
:1068D000400000202DE9F0410E46044600202062D1
:1068E0002046E168884730B3252805D0D4E9012146
:1068F0009047206A401CF2E7E1682046002788475D
:10690000050018D0A5F14100192802D820354FF410
:1069100000673246294620462760F9F721FC40B13E
:10692000012804D0F61D26F007060836D8E7361DE4
:10693000D6E72846DAE7206ABDE8F0812DE9F04184
:106940000646002410687529314616A510D0AFF30D
:106950000080002802DA404213A507E031688A0768
:1069600001D512A502E0490704D511A5012401E0D3
:10697000AFF3008000210A2206F1240709E0B0FBF2
:10698000F2FCB0FBF2F302FB1C00303078541846E6
:10699000491C0028F3D123462A463046BDE8F04181
:1069A00000F0B7B8000000002D0000002B00000030
:1069B0002000000040EA010310B59B070FD1042A14
:1069C0000DD310C808C9121F9C42F8D020BA19BABA
:1069D000884201D9012010BD4FF0FF3010BD1AB11F
:1069E000D30703D0521C07E0002010BD10F8013B74
:1069F00011F8014B1B1B07D110F8013B11F8014B9B
:106A00001B1B01D1921EF1D1184610BD02F0FF03ED
:106A100043EA032242EA024200F0E8B870477047B6
:106A20007047704753EA020C00F069802DE9F04B83
:106A30004FF00006002B1FBFB3FA83F503FA05F4ED
:106A400024FA05F65E4012BF1643B2FA82F502FA46
:106A500005F4C5F120051EBF22FA05FC44EA0C042A
:106A6000203556EA044C4FEA144418BF641C4FF01A
:106A700000084FF00009904271EB030C39D3002954
:106A800019BFB1FA81F701FA07F6B0FA80F700FAF8
:106A900007F6C7F120071EBF20FA07FC46EA0C06DE
:106AA0002037B6FBF4FCA7EB0507103F07F01F0BE0
:106AB000CBF120060CFA0BFB2CFA06F644BFB346CA
:106AC0000026202FA4BF5E464FF0000B5BEA060CA9
:106AD00008BF4FF0010B19EB0B09ABFB027C48EB35
:106AE0000608C01B06FB02CC0BFB03CC71EB0C01B0
:106AF000C1E70B46024641464846BDE8F08B13B558
:106B00004FF000004FF00001AFF30080BDE81C40E3
:106B100070472DE9F0470D4699469246044600F12C
:106B200024080168880604D5E06921F0100121607D
:106B300000E00120A84201DD471B00E00027A16919
:106B40007A1902EB0900081AA0612078C00602D465
:106B50002046AFF30080002608E0D4E901211AF8AE
:106B600006009047206A401C761C20624E45F4DBEC
:106B70002078C0060AD52046AFF3008006E0D4E9AD
:106B8000012130209047206A401C2062381EA7F166
:106B90000107F4DC07E0D4E9012118F8050090476B
:106BA000206A401C2062281EA5F10105F3DC204666
:106BB000AFF300802078000602D50220BDE8F08700
:106BC0000120FBE7074B70B50D467B4400F033F81E
:106BD0000446284600F042F810B14FF0FF3070BD77
:106BE000204670BD95B8FFFF4FF000020429C0F0A9
:106BF000128010F0030C00F03780CCF1040CBCF1D3
:106C0000020F18BF00F8012BA8BF20F8022BA1EB40
:106C10000C0100F029B85FEAC17C24BF00F8012B09
:106C200000F8012B48BF00F8012B704701694A1C8E
:106C300002610878704700B58FB0CDE901310021BD
:106C4000059105497944CDE9031011466846FFF7DF
:106C500041FE0FB000BD0000E5FFFFFF007B00F02C
:106C6000800070474FF0000200B5134694469646E8
:106C7000203922BFA0E80C50A0E80C50B1F120014F
:106C8000BFF4F7AF090728BFA0E80C5048BF0CC0FD
:106C90005DF804EB890028BF40F8042B08BF70475B
:106CA00048BF20F8022B11F0804F18BF00F8012BCD
:106CB0007047000000487047640500207546FFF7E4
:106CC000F9FFAE4605006946534620F007008546A9
:106CD00018B020B5F9F792FBBDE820404FF0000650
:106CE0004FF000074FF000084FF0000B21F00701B4
:106CF000AC46ACE8C009ACE8C009ACE8C009ACE8F7
:106D0000C0098D46704710B50446AFF30080204699
:106D1000BDE81040F9F736BA490050EAC12018BF63
:106D200004204A0D18BF40F0010040F2FF72B2EBA0
:106D3000515F08BF40F00200012808BF05207047DE
:106D40002DE9F0414F1E00EBC7010446D1E90001D7
:106D500015461E4637F006020DD02A46334600F08F
:106D60005BFC7F1E04EBC703D3E9002300F04CFA61
:106D700037F00602F1D1022F25D0042F13D0062FB1
:106D800018BFBDE8F0812A46334600F045FCD4E93F
:106D90000A2300F039FA2A46334600F03DFCD4E9D4
:106DA000082300F031FA2A46334600F035FCD4E9D6
:106DB000062300F029FA2A46334600F02DFCD4E9D8
:106DC000042300F021FA2A46334600F025FCD4E9DA
:106DD000022300F019FA2A46334600F01DFCD4E9DC
:106DE0000023BDE8F04100F00FBA012201F0E3B941
:106DF00000F00ABA024A0020110701F0DCB90000D5
:106E000001FDFFFF2DE9F84F04460D4621F000403B
:106E100000917349814211DC7249884201DC06D13C
:106E20002CB120462946BDE8F84FFFF7DEBF6E487B
:106E3000002DCCBF6D496E49BDE8F88F6D49814288
:106E400011DD6D498142D8BF4FF0FF366DDD204620
:106E50002946FFF761FF042808BFFFF7CBFF204654
:106E60002946BDE8F88F6549654F25F00045814208
:106E700033DD6449814219DD002632464FF08043FC
:106E80002046294600F0C0F980468A460122204665
:106E9000294601F090F900223B4600F0C7FC42462B
:106EA000534600F061FA04460D463EE001260022FA
:106EB000BA463B462046294600F0A6F980460F46D2
:106EC000002253462046294600F0B0FC42463B468D
:106ED00000F04AFA04460D4627E04B4981421BDD8B
:106EE000DFF828A10226002253462046294600F05A
:106EF00093FB00223B4600F087F980460F460022B4
:106F000053462046294600F091FC42463B4600F09D
:106F10002BFA04460D4608E0032622462B460020A5
:106F20003B4900F021FA04460D4622462B46104606
:106F3000194600F071FB8B46824602460B4600F074
:106F40006BFB07460246334888460B4606217844C9
:106F5000FFF7F6FE52465B4600F05EFB82462E4887
:106F60008B463A46434605217844FFF7E9FE3A4608
:106F7000434600F051FB02460B46002E5046594650
:106F80000CDA00F041F922462B4600F045FB01B037
:106F900022462B46BDE8F04F00F03CBC00F034F92F
:106FA00022462B4600F038FB1C4A7A4402EBC6030B
:106FB000D3E9002300F03AFC22462B4600F036FCD1
:106FC000174A7A4402EBC603D3E9002300F022FCFF
:106FD000009A002AB8BF81F00041BDE8F88F000098
:106FE000000010440000F07F182D4454FB21F93FAD
:106FF000FB21F9BF0000DC3F0000203E0000F33F12
:107000000000F03F0000E63F008003400000F83F32
:107010000000F0BF062A0000C42900006229000019
:107020002A2900002DE9F04D9446CCF1000423F00C
:1070300000464CEA0404524F46EAD4749A46884605
:1070400021F00042BC4206D8454240EA050442EA2B
:10705000D474BC4204D9BDE8F04D6246FFF7C8BE07
:10706000AAF14055A5F17F6555EA0C040BD0022426
:1070700004EAAA74434DDFF810E144EAD87452EAF6
:10708000000B04D00CE0BDE8F04DFFF7BBBE002CB8
:1070900014BF012CBDE8F08D022C30D0032C32D06F
:1070A00056EA0C0B0AD0BE4220D1BA4209D126F0D2
:1070B000804622F080423346114617E000291ADB51
:1070C00025E0DFF8C8B0FB44002C04BFDBE9000179
:1070D000BDE8F08D012C02BFDBE9000181F0004129
:1070E000BDE8F08D022C0AD0032C0CD0BA4212D18C
:1070F000B8F1000F0BDA23482549BDE8F08D28468A
:107100002449BDE8F08D28467146BDE8F08D1D4844
:107110002149BDE8F08D921B12153C2AC4BF1948C5
:107120001D490EDCBAF1000FBEBF12F13C0F00206A
:10713000014606DB624600F017F921F00041FFF737
:1071400061FE002C08BFBDE8F08D012C04BF81F06A
:107150000041BDE8F08D114A114B022C07D000F020
:1071600065FB2A46BDE8F04D0A4B00F05FBB00F01E
:107170005DFB2A46BDE8F04D064B00F04BBB00001E
:107180000000F07F182D4454FB2109C0BE280000E8
:10719000FB21F9BFFB210940FB21F93F075C1433B8
:1071A00026A6A13C21F00042A2F16052B2F5801F58
:1071B00001F0004328BFD2F17F6C0BD95FEA001CBD
:1071C00043EAC20242EB507018BF704728BF20F05C
:1071D00001007047B2F5801FBCBF184670474FEAE8
:1071E000410C1CF5001F02D2084600F0FCBE70B531
:1071F00000F0BCFA00000089FFF7F6BF4FF0004036
:10720000A0F580007047000010B591EA030F48BF59
:1072100083F0004300F11283841A71EB030C05D252
:10722000121943EB0C03001B61EB0C01DFF824E1A6
:107230004FEA1154A4EB135C1EEA430F18BF9EEAF9
:10724000445F73D023EA0E03DCF1200E21EA0451DF
:1072500043F4801332D322FA0CFE10EB0E0023FA13
:107260000CFE41EB0E01CCF1200E03FA0EFE10EBEA
:107270000E0051F10001B1F5801FCCF1200E32D289
:1072800001EB045112FA0EF2BDE8104058BF7047EE
:10729000401C38BF5FEA420218BF7047002814BF85
:1072A00020F0010041F100014FEA410313F5001FF6
:1072B00038BF7047A1F1C04100F0A6BA012A43EBE4
:1072C0000302ACF1200CDCF11F0E32BF4FF0000EB8
:1072D00023FA0CF310EB030041EB0451B4EB115F04
:1072E000D0D0A1EB045101F5801149085FEA3000CC
:1072F00001EB04510ED350F1000038BF12FA0EFE1C
:1073000008D1BDE81040C9E7401C38BF5FEA42021F
:10731000CAD1C3E7BDE810404FEA410313F5001F8F
:1073200038BF7047A1F1C04100F06EBA9EEA445FD9
:1073300008D011EA5E0FBDE8104004BF01F0004123
:1073400000207047BDE8104070B500F00FFA00BF94
:1073500064FBBE3E0000E0FF02494FF0000000F079
:10736000F8BE00BF0000F87F2DE9C04130B4DFF85F
:10737000A0C23CEA111418BF3CEA131400F0EC80E0
:1073800081EA03051CEA111444EAD57418BF1CEA0B
:10739000131500F0C780A4EB05044FF0004545EA43
:1073A000C12145EAC32341EA505143EA525304F153
:1073B0007F74994204F500344FEAC0204FEAC2229C
:1073C00008BF904200F09C804FEA13650FF2401610
:1073D000765D4FEA134506FB05F7C7F1807706FB9C
:1073E00007F74FEAD737A7FB03687642C8F580381E
:1073F000A7FB06CE38BFA8F1010807FB08E64FF04F
:10740000000EA6FB028CE6FB03CEDCF1000CCEF1F5
:10741000004E38BFAEF1010EA6FB0C584FF000072E
:107420004FF00005E6FB0E87A1FB08C6A0FB07CEC8
:1074300016EB0E0645F10005E1FB076515F1E04E80
:107440007EBFA4F580345FEA46066D4116F18007E1
:1074500045F100054FEA17274FEA066647EA056738
:10746000A6F1DE46B6F1805F4FEA15251FD93846F2
:1074700024F0010C05EBC471BCF1FE6F01EB0C11A3
:1074800002D8F0BCBDE8008124425CBF01F5801E3B
:107490009EEAC47F02D4F0BCBDE80081244238D407
:1074A000F0BCA1F1C041BDE8004100F0ADB94FEA28
:1074B000D22242EA43524FEAD323A7FB02864FEA85
:1074C000D02040EA415007FB03661EEA0E0F4FEA48
:1074D000D12105FB026658BFA6EB0056B6EB00565D
:1074E0004FEA520E4EEAC37E18EB0E0E56EB530EC9
:1074F000BDD518EB02085E417F1C55F10005B6E7CB
:107500004FF480154FF000074FF000064FF00008D1
:10751000ADE7F0BC4FF0000001F1C04101F00041C7
:10752000BDE8008111EA0C1F0CEA131500D00CE035
:1075300013EA0C1F00F025804FF00000F0BC81EA38
:10754000030101F00041BDE80081F0BCBDE800414D
:1075500081EA030100F058B9F0BCBDE8004170B504
:1075600000F004F9097EFC3E00F007B881EA03014F
:107570004FF0000001F00041704781EA030100F084
:1075800043B9F0BCBDE800414FF00000214970470D
:10759000FFFDFBF9F7F5F4F2F0EEEDEBE9E8E6E4D8
:1075A000E3E1E0DEDDDBDAD8D7D5D4D3D1D0CFCD5F
:1075B000CCCBCAC8C7C6C5C4C2C1C0BFBEBDBCBB98
:1075C000BAB9B8B7B6B5B4B3B2B1B0AFAEADACAB93
:1075D000AAA9A8A8A7A6A5A4A3A3A2A1A09F9F9E6D
:1075E0009D9C9C9B9A99999897979695959493931F
:1075F000929191908F8F8E8E8D8C8C8B8B8A8989B6
:107600008888878786858584848383828281818038
:107610000000FF070000F87FDFF848C170B51CEAE2
:10762000111E1EBF1CEA13159EEA0C0F95EA0C0FE3
:1076300000F06F8081EA030423EA4C134EEAD47E03
:1076400021EA4C1141F4801143F48013AE44A1FBB4
:10765000024CA0FB0365AEF17F7E361955EB0C059D
:10766000A1FB034C4CF10003A0FB021C16EB0C0623
:10767000654153F10003094218BF46F0010613F4B7
:10768000007F0BD14FEA03314FEA0530340341EA62
:10769000155140EA16506FF003020AE04FEAC32189
:1076A0004FEAC520F40241EA555140EA56506FF0C6
:1076B000020202EB2E4201EB025585EACE710AD09E
:1076C0005FEA440C18BF24F0004450F1000041F17F
:1076D000000120EAD47040F2FE7C624500D270BD09
:1076E000A84214BF4FF080444FF04044002E08BF22
:1076F0000024BEF1806FA8BFA1F1C041BDE8704079
:1077000080F282804FF0000001F1C04101F00041A1
:1077100070479EEA0C0F0CEA131518BF95EA0C0F80
:1077200006D04FF0000081EA030E0EF0004170BD5C
:1077300000F01CF88900013E00F007B800F009B81D
:107740004FEA430C5FEA5C5C08D081EA030100F079
:107750005BB84FEA410C5FEA5C5CF6D14FF0000089
:10776000014970470000FF070000F87F0EF1020E8C
:107770002EF0030E5EF8046B364205D4012A43EB6B
:10778000030515F5001F12D8012841EB010C1CF56B
:10779000001F0CD80ED14FEAD17C15F5001F0CEB61
:1077A0004C0C0CF1020C08BF4CEBD37C04E04FF006
:1077B000080C01E04FEAD37C0CEB4C0526FA05F6E9
:1077C00006F00706B6F1040C06D20EEB860CBDE8F7
:1077D00070404CF0010C6047DFE80CF0090B02022E
:1077E0004FF000414FF00000A1F5002170BD194697
:1077F0001046012851EB010418BFD4F5001484BFD2
:10780000002001F0004170BD0808A0F500114FEA0A
:107810003101704791EA030F10B581F000413FF547
:10782000FBAC83F0004300F009B8000010B591EA0A
:10783000030F48BF83F000433FF5EEAC841A71EBB1
:10784000030C07D212198CF0004C43EB0C03001B05
:1078500061EB0C01DFF8A4E14FEA1154A4EB135CD7
:107860001EEA430F18BF9EEA445F00F0B08023EA8F
:107870006E03524221EA0451C3EB6E0338BF5B1E14
:10788000DCF1200E25D322FA0CFE10EB0E0043FA99
:107890000CFE41EB0E01CCF1200E03FA0EFE10EBB4
:1078A0000E0051F10001CCF1200E29D412FA0EF293
:1078B00001EB0451BDE8104058BF7047401C1CBF8D
:1078C000B2F1004F704700280CBF491C20F00100A6
:1078D000704712EB020E43EB030218BF4FF0010E8C
:1078E0004EEA4202ACF1200CDCF11E0E54D943FAF0
:1078F0000CFE10EB0E0051F1FF31CCF11E0ED5D570
:107900000EF1010E12FA0EFE404141EB010101EBB6
:10791000445C5FEA5C5C10D910EBDE7001EB045153
:1079200038BFBEF1004FBDE8104018BF70470028B7
:107930000CBF491C20F00100704730D24FEAD42C14
:1079400011F5001124F400641BD0B1FA81F20B3A56
:10795000A41AA41ED2F12003914030FA03F3194374
:10796000904001EBCC71002C01EB0451BDE81040BC
:10797000A8BF704701F1C0414FF0000001F0004185
:107980007047B0FA80F310FA03F100D110BDE41A89
:10799000173C4805C90AE4E701EB045110BD491042
:1079A00001EB0451BDE810404FEA300002E04FF017
:1079B000000170474A0008BF0042F8D0B2F5001F2E
:1079C00028BF704701F000414FF0000070479EEA69
:1079D000445F07D011EA5E0FBDE8104004BF0021EC
:1079E00000207047BDE8104070B5FFF7BFFE00BF34
:1079F00040DFF63E83F00041104670470000E0FF94
:107A000043004FEAD30C4FEA3C0C43401FBF4007F2
:107A10000CF1605113F0FE4F70471CF0006F03D162
:107A200000200CF0004170470CF0004343EA507016
:107A300010B540EACC0000F090FA00BF00000092C0
:107A40004FEA0001FFF7E0BE4FF000414FF00000A9
:107A5000A1F500217047000090EA010F48BF81F0B6
:107A6000004100F10883421A3CBF801A89184FEA8E
:107A7000D0524FF07F4C1CEA410FA2EBD15318BFFC
:107A80009CEA026F00F03B804FF0004C4CEA002073
:107A90004CEA012121FA03FC10EB0C0C1ED202F17E
:107AA000FF325FEA1C2040EBC25038BF70471CF029
:107AB0007F0F4FEA400C18BFBCF17F4F38BF7047B3
:107AC000C3F12003994008BF20F00100BCF17F4FB3
:107AD00038BF7047A0F1C04000F085BA4FEA3C00C3
:107AE000000A40EBC25028BF1CF0FF0F4FEA400CC9
:107AF000E6D018BFBCF17F4F38BF7047EAE79CEA79
:107B0000026F05D010EA5C0F08BF00F0004070471C
:107B100010B500F022FA00BF64FBBE3E401058BF13
:107B2000C0F14040491058BFC1F140418142EFF3DC
:107B3000008070474FF47F0C1CEAD0121EBF1CEA75
:107B4000D11392EA0C0F93EA0C0F00F0858090EAB3
:107B5000010F48BF42F4807240F4000C41F4000071
:107B60002CF07F4120F07F4000B58142A2EB030260
:107B70000FF2081CACEB504EC0F100009EF800E084
:107B80004FEA4E0E00FB0EFC38BF49004FEA2C1C9A
:107B900002F5FA020CFB0EF34FEACE1E4FEA112C4F
:107BA0004FEAC1210EEB635E42EB22420EFB0CFC5E
:107BB0004FEA1C5300FB03114FEA112C4FEA01312D
:107BC0000EFB0CFC4FEADC4C00FB0C11C14228BF41
:107BD00009184CEB03335DF804EB10EB410143EB68
:107BE000C250B2F57C0F38BF704729D512F0F00FA4
:107BF0001CBF00F1C04000F000407047008182834C
:107C00008485868788898B8C8D8E8F9192939596AB
:107C100097999A9C9D9FA0A2A3A5A7A8AAACAEB035
:107C2000B2B3B5B7B9BCBEC0C2C5C7C9CCCED1D43A
:107C3000D7D9DCDFE2E6E9ECF0F3F7FAFE0000006A
:107C40004FEA400C0CF1807CBCF17E4F28BF70479E
:107C5000B0F1C04000F0C7B990EA010F0CEAD113AF
:107C600048BF42F48072624538BF634507D213F4BF
:107C70007F0F16D080EA010000F00040704710B579
:107C800000F06BF9097EFC3E00F005B880EA0100C7
:107C900000F00040704780EA010000F0004000F072
:107CA000A2B912F47F0F04BF0248704780EA0100B6
:107CB00000F099B90000C07F50EA010C00F1138078
:107CC0001CF5000F58BFBCF5000F01D48842704767
:107CD00007D710F5000F58BF11F5000F15D48842D3
:107CE0007047894270471CF5000F04D5BCF5000FA2
:107CF000F7D5814270474FF0807C1CEB400F38BFB6
:107D00001CEB410F01D28142704710B500F025F9FC
:107D1000922449004FF000504FF08051FFF7FEBE13
:107D200041000B0ED3F19E0208D950F400034FEA34
:107D3000032323FA02F048BF4042704710B500F019
:107D40000CF900BF49922480002070476FF0004278
:107D500082EA200070470000C10DD1F19E0206DBCF
:107D60004FEA002343F0004323FA02F07047004239
:107D700007D54FEA4001B1F1FE4F02D24FF00000AB
:107D8000704710B500F0E9F8499224800020704750
:107D90006FEA20007047000010F0004148BF4042E9
:107DA000B0FA80F310FA03F2C3F19D030BD051EA4D
:107DB000C35101EB1220530638BF704700F1010098
:107DC00008BF20F001007047B0FA80F310FA03F208
:107DD000C3F19D030AD0D90501EB1220530638BF29
:107DE000704700F1010008BF20F00100704700005B
:107DF00050EA010C00F113801CF5000F58BFBCF5D0
:107E0000000F01D48842704707D710F5000F58BF04
:107E100011F5000F15D488427047894270471CF550
:107E2000000F04D5BCF5000FF7D5814270474FF025
:107E3000807C1CEB400F38BF1CEB410F01D281420C
:107E4000704710B500F089F8922449004FF00050B7
:107E50004FF08051FFF762BE4FF47F0C1CEAD01246
:107E60001EBF1CEAD11392EA0C0F93EA0C0F00F02C
:107E7000478090EA010F48BF42F480724FF0004CF7
:107E80004CEA00204CEA012102EB0302A0FB0113A3
:107E9000A2F50002002918BF43F001035B0028BFD0
:107EA0004FEA330342EB22425FEA132C4CEBC25001
:107EB0002EBFBCEB436FB2F57C0F70474FEA036CEB
:107EC000BCF1004F08BF20F00100B2F57C0F38BFB5
:107ED00070470BD582F0FF0212F5803FC8BF704794
:107EE00000F1C040D8BF00F00040704700F5000C22
:107EF0005FEA4C0C48BF7047B0F1C04000F073B867
:107F000090EA010F0CEAD11348BF42F48072624537
:107F100038BF634504D280EA010000F0004070479A
:107F200010B500F01AF800BF8900013E00F007B854
:107F300000F009B85FEA410C5FEA1C6C08D080EAE7
:107F4000010000F050B85FEA400C5FEA1C6CF6D10B
:107F50004FF00040A0F5800070470EF1020E2EF0A9
:107F6000030E5EF8044B244204D44FEA4102B2F1FE
:107F70007F4F11D84FEA4003B3F17F4F0CD80ED199
:107F80004FEAD07CB2F17F4F0CEB4C0C0CF1020CA1
:107F900008BF4CEBD17C04E04FF0080C01E04FEA45
:107FA000D17C0CEB4C0324FA03F404F00704B4F185
:107FB000040C06D20EEB840CBDE810404CF0010C12
:107FC0006047DFE80CF0070802024FF00040A0F520
:107FD000800010BD0846420018BFD2F1807288BFF1
:107FE00000F0004010BDFF2141EAD050C0057047AD
:107FF00051EA000C00F113801CF5000F58BFBCF5CE
:10800000000F01D48142704707D711F5000F58BF08
:1080100010F5000F15D481427047894270471CF556
:10802000000F04D5BCF5000FF7D5884270474FF01C
:10803000807C1CEB410F38BF1CEB400F01D2884203
:10804000704780EA010081EA000180EA0100FFF741
:10805000F8BE80F0004090EA010F7FF504AD81F09A
:10806000004100F008B8000090EA010F48BF81F01D
:1080700000413FF5F8AC421A04D882F00042A0EB70
:10808000020011444FEAD0524FF07F4C1CEA410FDE
:10809000A2EBD15318BF9CEA026F4AD04FF0004CBC
:1080A0004CEA00204CEA012121FA03FCB0EB0C0C55
:1080B0000FD412F0FE0F36D05FEA4C001DD500122F
:1080C00040EBC25038BF70471CF03F0F18BF7047DD
:1080D0000BE0A2F101025FEA1C2040EBC25038BF66
:1080E00070471CF07F0F18BF7047C3F12003994001
:1080F00014BF401E20F00100704780084FEA122391
:1081000008BF7047B0FA80FCA2EB0C02CCF1280C3F
:1081100060FA0CF093EA122F04BF00EBC2507047D4
:108120004FEAC3707047130A5FEADC1008BF70475C
:10813000F6E79CEA026F04D010EA5C0F08BF00204B
:10814000704710B5FFF709FF40DFF63E81F00040B1
:1081500070470CF00F03092B08BF082000F059806E
:108160000A2B0BD0082B18BF704708BF1CF0400F1C
:108170000AD04FF000004FF0000170471CF0400F94
:1081800018BF4FF0004070471CF0100F08D020F0CF
:10819000704300F07F4242EAD3014FEA43707047D8
:1081A00000F0604021F07F4242EA000201F07F408F
:1081B00040EA727070474FF0FF0C4CF4E06C1CEA20
:1081C00011531CBF9CEA030C9445C2BFDA4201EB79
:1081D00002517047002B0DD0BCF1000F0FD0002AC8
:1081E00001F00041A4BF41F0E04141F07F614FF058
:1081F0000000704701F000414FF00000704750EA66
:1082000001334FF09B0C18BF4CF0806C7FF4A4A896
:1082100070471CF4801F11D01CF4E02F03D06FEACC
:10822000CC31490070474FF04050EFF3008222F00C
:10823000704242EA000282F3008870474FF000006B
:108240007047000000000000000000000000000077
:1082500000003F400000000000000000300040002F
:1082600030004000000009000BC03D000BC03D0085
:10827000090018C024407FE022403180000018002F
:1082800024C01B000D803240018003801C40274029
:108290001C8007400040100060000000000000004B
:1082A00000000000000000001F802040402000006F
:1082B000402020401F8000000000090006001F80B1
:1082C000060009000000040004003F8004000400D0
:1082D000000000100060000000000000000004002A
:1082E000040004000400040000000000004000003E
:1082F000000000000000002001C00600380040001F
:1083000000001F802040204020401F80000000000F
:1083100010403FC000400000000018C02140224033
:1083200024401840000010802040244024401B803E
:10833000000002000D0011003FC0014000003C8021
:10834000244024402440238000001F8024402440F7
:108350003440038000003000200027C03800200097
:1083600000001B802440244024401B8000001C008F
:1083700022C0224022401F80000000000000084070
:108380000000000000000000000004600000000089
:108390000000000004000A00110020804040090095
:1083A0000900090009000900000000004040208089
:1083B00011000A00040018002000234024001800C7
:1083C00000001F802040274029401F40000000403F
:1083D00007C039000F0001C0004020403FC02440CA
:1083E00024401B8000001F8020402040204030801F
:1083F000000020403FC0204020401F80000020405F
:108400003FC024402E4030C0000020403FC02440E8
:108410002E00300000000F001080204022403380EA
:10842000020020403FC0040004003FC02040204024
:1084300020403FC02040204000000060202020203D
:108440003FC02000200020403FC024400B0030C02F
:10845000204020403FC020400040004000C03FC0BE
:108460003C0003C03C003FC0000020403FC00C4027
:1084700023003FC020001F802040204020401F805C
:10848000000020403FC024402400180000001F804E
:108490002140214020E01FA0000020403FC0244098
:1084A000260019C0004018C02440244022403180DA
:1084B0000000300020403FC020403000000020007D
:1084C0003F80004000403F80200020003E0001C06F
:1084D000070038002000380007C03C0007C0380003
:1084E0000000204039C0060039C0204000002000B4
:1084F000384007C0384020000000304021C02640EE
:10850000384020C00000000000007FE040204020F4
:108510000000000070000C0003800040000000001C
:10852000402040207FE000000000000020004000CC
:1085300020000000000000100010001000100010CB
:1085400000100000000040000000000000000000DB
:1085500002800540054003C0004020003FC00440A9
:1085600004400380000000000380044004400640F3
:10857000000000000380044024403FC00040000091
:1085800003800540054003400000000004401FC078
:10859000244024402000000002E005500550065011
:1085A000042020403FC00440040003C000400000FD
:1085B000044027C00040000000000010001004101C
:1085C00027E00000000020403FC00140070004C039
:1085D0000440204020403FC000400040000007C051
:1085E000040007C0040003C00000044007C00440AA
:1085F000040003C0004000000380044004400380E6
:108600000000041007F00450044003800000000044
:1086100003800440045007F00010044007C00240EB
:10862000040004000000000006400540054004C0AE
:108630000000000004001F8004400040000004000F
:1086400007800040044007C000400400070004C049
:10865000018006000400060001C0070001C00600FA
:108660000000044006C0010006C0044000000410E1
:10867000071004E00180060004000000044005C06B
:108680000640044000000000000004007BE04020A1
:108690000000000000000000FFF0000000000000EB
:1086A00040207BE00400000000004000800040000B
:1086B000200020004000000000000000000000003A
:1086C0000000000000000000000000001FCC000CB3
:1086D00000000000000000000800300060000800FA
:1086E000300060000000022003FC1E20022003FC7A
:1086F0001E200220000000000E1811043FFF10840D
:108700000C78000000000F0010840F3800C00778BC
:1087100018840078000000780F8410C411240E988B
:1087200000E40084000808006800700000000000F9
:1087300000000000000000000000000007E0181822
:10874000200440020000000040022004181807E046
:108750000000000000000240024001800FF0018094
:108760000240024000000080008000800FF800807E
:108770000080008000000001000D000E00000000DD
:1087800000000000000000000080008000800080E9
:108790000080008000800000000C000C0000000041
:1087A00000000000000000000006001800600180CA
:1087B000060018002000000007F00808100410044C
:1087C000080807F000000000080408041FFC00046B
:1087D00000040000000000000E0C101410241044CF
:1087E00011840E0C000000000C1810041104110478
:1087F00012880C700000000000E00320042408240C
:108800001FFC0024000000001F98108411041104B4
:10881000108810700000000007F00888110411048F
:1088200018880070000000001C00100010FC1300ED
:108830001C001000000000000E3811441084108449
:1088400011440E38000000000700088C104410444A
:10885000088807F00000000000000000030C030C73
:108860000000000000000000000000010106000000
:108870000000000000000000008001400220041001
:10888000080810040000022002200220022002201A
:10889000022002200000000010040808041002203A
:1088A00001400080000000000E001200100C106C4F
:1088B00010800F00000003E00C1813E4142417C408
:1088C000082807D000000004003C03C41C400740F7
:1088D00000E4001C000410041FFC11041104110426
:1088E0000E880070000003E00C181004100410043F
:1088F00010081C10000010041FFC100410041004C9
:10890000080807F0000010041FFC1104110417C42C
:1089100010040818000010041FFC1104110017C0F7
:1089200010000800000003E00C18100410041044AC
:108930001C780040000010041FFC108400800080A0
:1089400010841FFC10040000100410041FFC10040D
:1089500010040000000000030001100110011FFEC0
:1089600010001000000010041FFC110403801464A8
:10897000181C1004000010041FFC10040004000464
:108980000004000C000010041FFC1F0000FC1F006E
:108990001FFC1004000010041FFC0C04030000E086
:1089A00010181FFC100007F0080810041004100431
:1089B000080807F0000010041FFC108410801080CD
:1089C00010800F00000007F0081810241024101C5D
:1089D000080A07F2000010041FFC1104110011C066
:1089E00011300E0C000400000E1C110410841084C1
:1089F00010441C3800001800100010041FFC100464
:108A000010001800000010001FF8100400040004FB
:108A100010041FF8100010001E0011E0001C007070
:108A200013801C0010001FC0103C00E01F0000E07D
:108A3000103C1FC000001004180C163401C001C007
:108A40001634180C100410001C00130400FC13044E
:108A50001C00100000000804101C10641084130493
:108A60001C04101800000000000000007FFE4002FF
:108A7000400240020000000030000C000380006053
:108A8000001C0003000000004002400240027FFE84
:108A90000000000000000000000020004000400036
:108AA0004000200000000001000100010001000161
:108AB0000001000100010000400040002000000013
:108AC000000000000000000000980124014401445F
:108AD000014400FC000410001FFC00880104010494
:108AE000008800700000000000700088010401048C
:108AF00001040088000000000070008801040104E7
:108B000011081FFC0004000000F801440144014466
:108B1000014400C800000000010401040FFC11041E
:108B2000110411001800000000D6012901290129B3
:108B300001C90106000010041FFC008401000100AF
:108B4000010400FC000400000104190419FC0004E5
:108B500000040000000000000003000101011901F1
:108B600019FE0000000010041FFC0024004001B4A6
:108B7000010C010400000000100410041FFC00049C
:108B8000000400000000010401FC0104010001FCDC
:108B90000104010000FC010401FC0084010001004B
:108BA000010400FC0004000000F8010401040104B9
:108BB000010400F80000010101FF00850104010427
:108BC00000880070000000000070008801040104AB
:108BD000010501FF00010104010401FC00840104FE
:108BE000010001800000000000CC012401240124C8
:108BF00001240198000000000100010007F80104B1
:108C0000010400000000010001F800040004000459
:108C1000010801FC0004010001800170000C00103B
:108C200001600180010001F0010C003001C0003042
:108C3000010C01F0010000000104018C00740170BE
:108C4000018C01040000010101810171000E001876
:108C500001600180010000000184010C0134014425
:108C60000184010C00000000000000000000010071
:108C70003EFC400240020000000000000000FFFF38
:108C80000000000000000000400240023EFC010025
:108C90000000000000000000600080008000400034
:108CA000400020002000000068000004760054010D
:108CB000F7FD000175191A0C6A231B1C1F20727422
:108CC000433B4138393A6B6C376F06246D6E700048
:108CD00083000000000800000001001832000500B9
:108CE000000020410000D242295C0F3E9A99993E33
:108CF0003333733F295C0F3E0000700000000024F6
:108D0000000000020003000000650054FFEF0000B7
:108D1000FA80000B12820001030C30C30E8C8CE928
:108D200014D5400213710F8E3883F8833000F88316
:108D3000258EF8833000F883FFFFFFFF0FFEA9D6D2
:108D4000240004001A8279A10000003CFFFF00000B
:108D50000010000038836FA2003E03304000000086
:108D600002CAE3093E80000020000000000000006D
:108D70004000000060000000000C0000000C186EB5
:108D8000000006920A16C0DFFFFF0256FD8CD37763
:108D9000FFE1C496E0C5BEAA00000000FFFF0B2B58
:108DA00000001657000003594000000000001DFAA3
:108DB00000026C1D000000003FFFDFEB003EB3B679
:108DC000000D227800002F3C00000000001942B581
:108DD000000039A20000B365D90E9FC91DCF4C34E5
:108DE00030000000500000003BB67AE8006400004C
:108DF00000C8000000000000100000001000FA92FF
:108E00001000225E000D229F0001000000320000D1
:108E1000FF46000063D400001000000004D60000EC
:108E200004CC000004CC00000000107200000040E0
:108E3000000000000000000000060002000500071E
:108E400000000000006400000000000000000005B9
:108E50000005006400200000000000000000000089
:108E6000000040000000030000000032F8980000FD
:108E7000FF650000830F0000FF9BFC000000000066
:108E800000000000000000000000000000000000E2
:108E900000000000000000000000000000000000D2
:108EA000000000000000100040000000000000066C
:108EB0000000B26A000200000001FB8300680000AD
:108EC00000D9FC007CF1FF83000000000065000079
:108ED000006403E800640028000000250000000092
:108EE00016A000000000100000001000002F00007D
:108EF000000001F40000100000280000FFFF458181
:108F0000FFFFFA72000000000000000000440005AE
:108F10000005BAC6004778A200000001000000006A
:108F200000000600000000140000254D002F706DA9
:108F3000000005AE000C02D00000000000000000A0
:108F40000000000000000000001B00000000000006
:108F500000000000000000000064000000080000A5
:108F60000000000000000000000000000000000001
:108F700000000000000000000000000000000000F1
:108F800000000000000000000000000000000000E1
:108F900000000000000000000000000000000000D1
:108FA00000000000000000000000000000000000C1
:108FB0000000000000000000001B00000000000096
:108FC00000000000000E000E00000AC700040000B0
:108FD00000000032FFFFFF9C00000B2B000000028E
:108FE0000000000100000064FFE500000000000038
:108FF0000000000000000000000000010000000070
:10900000000100000000000000018000000180005D
:1090100000018000002426D30000000000000000B2
:10902000000600100096003C000000000000000058
:1090300000000000000000000C0A4E68CDCF770948
:1090400050166759C619CE820000000000000000CB
:109050000000000000000000000000000000000010
:1090600017D784000300000000000000000000008B
:10907000C7938F9D1E1B1C190000000000000000FC
:1090800000000000000000000000000000000000E0
:1090900002031885000040000000000300000003E8
:1090A0000000000000000000400000000000000080
:1090B00000000000000000000000000000000000B0
:1090C00000000000000000000000000000000000A0
:1090D000000000000000000000000000677DDF7E4F
:1090E00072902E554CF6E68800000000000000004B
:1090F0000000000000000000D8DCB4B8B0D8B9AB64
:10910000F3F8FAB3B7BB8E9EAEF132F51BF1B4B8EB
:10911000B08097F1A9DFDFDFAADFDFDFF2AAC5CDDC
:10912000C7A90CC92C97F1A989264666B28999A9C5
:109130002D557DB0B08AA896365676F1BAA3B4B252
:1091400080C0B8A89711B28398BAA3F0240844103D
:109150006418B2B9B49883F1A329557DBAB5B1A307
:109160008393F0002850F5B2B6AA839328547CF17B
:10917000B9A3829361BAA2DADEDFDB819AB9AEF5D8
:10918000606870F1DABAA2DFD9BAA2FAB9A3829202
:10919000DB31BAA2D9BAA2F8DF85A4D0C1BBAD83B6
:1091A000C2C5C7B8A2DFDFDFBAA0DFDFDFD8D8F1E2
:1091B000B8AAB38DB4980D355DB2B6BAAF8C961916
:1091C0008F9FA70E161EB49AB8AA872C547CBAA4F7
:1091D000B08AB691325676B28494A4C808CDD8B875
:1091E000B4B0F19982A82D557D98A80E161EA22C18
:1091F000547C92A4F02C5078F184A898C4CDFCD86B
:109200000DDBA8FC2DF3D9BAA6F8DABAA6DED8BAD7
:10921000B2B68696A6D0F3C841DAA6C8F8D8B0B4DC
:10922000B882A892F52C548898F135D9F418D8F161
:10923000A2D0F8F9A884D9C7DFF8F883C5DADF69C6
:10924000DF83C1D8F40114F1A8824EA884F311D1B0
:1092500082F5D992289788F109F41C1CD884A8F3C8
:10926000C0F9D1D99782F129F40DD8F3F9F9D1D900
:1092700082F4C203D8DEDF1AD8F1A2FAF9A88498E2
:10928000D9C7DFF8F8F883C7DADF69DFF883C3D816
:10929000F40114F198A8822EA884F311D182F5D993
:1092A00092509788F109F41CD884A8F3C0F8F9D13A
:1092B000D99782F149F40DD8F3F9F9D1D982F4C4E0
:1092C00003D8DEDFD8F1AD8898CCA809F9D982920D
:1092D000A8F57CF1883ACF944A6E98DB6931DAAD13
:1092E000F2DEF9D88795A8F221D1DAA5F9F417D9D9
:1092F000F1AE8ED0C0C3AE82C684C3A88595C8A582
:1093000088F2C0F1F4010EF18E9EA8C63E56F554C7
:10931000F18872F40115F19845856EF58E9E0488EA
:10932000F142985A8E9E068869F4011CF1981E112C
:1093300008D0F504F11E970202983625DBF9D9858D
:10934000A5F3C1DA85A5F3DFD88595A8F309DAA5D9
:10935000FAD88292A8F578F1881A849F26889821F5
:10936000DAF41DF3D8879F39D1AFD9DFDFFBF9F4E9
:109370000CF3D8FAD0F8DAF9F9D0DFD9F9D8F40B30
:10938000D8F3879F39D1AFD9DFDFF41DF3D8FAFCCA
:10939000A869F9F9AFD0DADEFAD9F88F9FA8F1CC35
:1093A000F398DB45D9AFDFD0F8D8F18F9FA8CAF387
:1093B0008809DAAF8FCBF8D8F2AD978D0CD9A5DF3D
:1093C000F9BAA6F3FAF412F2D8950DD1D9BAA6F3E8
:1093D000FADAA5F2C1BAA6F3DFD8F1BAB2B6869628
:1093E000A6D0CAF349DAA6CBF8D8B0B4B8D8AD84C1
:1093F000F2C0DFF18FCBC3A8B2B68696C8C1CBC38B
:10940000F3B0B48898A821DB718D9D71859521D921
:10941000ADF2FAD88597A828D9F408D8F28D29DAC0
:10942000F405D9F285A4C2F2D8A88D9401D1D9F45B
:1094300011F2D88721D8F40AD8F28498A8C801D1AB
:10944000D9F411D8F3A4C8BBAFD0F2DEF8F8F8F81D
:10945000F8F8F8F8D8F1B8F6B5B9B08A95A3DE3CBB
:10946000A3D9F8D85CA3D9F8D87CA3D9F8D8F8F94F
:10947000D1A5D9DFDAFAD8B18530F7D9DED8F830FE
:10948000ADDADED8F2B48C99A32D557DA083DFDF51
:10949000DFB591A0F629D9FBD8A0FC29D9FAD8A02C
:1094A000D051D9F8D8FC51D9F9D879D9FBD8A0D066
:1094B000FC79D9FAD8A1F9F9F9F9F9A0DADFDFDFF7
:1094C000D8A1F8F8F8F8F8ACDEF8ADDE8393AC2C50
:1094D000547CF1A8DFDFDFF69D2CDAA0DFD9FADBC0
:1094E0002DF8D8A850DAA0D0DED9D0F8F8F8DB559E
:1094F000F8D8A878DAA0D0DFD9D0FAF8F8F8F8DBF5
:109500007DF8D89CA88CF530DB38D9D0DEDFA0D030
:10951000DEDFD8A848DB58D9DFD0DEA0DFD0DED828
:10952000A868DB70D9DFDFA0DFDFD8F1A888902C36
:10953000547C98A8D05C38D1DAF2AE8CDFF9D8B080
:1095400087A8C1C1B188A8C6F9F9DA36D8A8F9DA6E
:1095500036D8A8F9DA36D8A8F9DA36D8A8F9DA363A
:10956000D8F78D9DADF818DAF2AEDFD8F7ADFA3046
:10957000D9A4DEF9D8F2AEDEFAF983A7D9C3C5C7FC
:10958000F1889BA77AADF7DEDFA4F8849408A7974B
:10959000F300AEF29819A488C6A39488F632DFF2DD
:1095A0008393DB09D9F2AADFD8D8AEF8F9D1DAF380
:1095B000A4DEA7F1889B7AD8F38494AE19F9DAAACD
:1095C000F1DFD8A881C0C3C5C7A39283F628ADDE5A
:1095D000D9F8D8A350ADD9F8D8A378ADD9F8D8F830
:1095E000F9D1A1DADEC3C5C7D8A18194F818F2B0C9
:1095F00089ACC3C5C7F1D8B8B4B09786A8319B066B
:109600009907AB9728889BF00C201440B0B4B8F0B1
:10961000A88A9A285078B79BA82951792470594470
:109620006938644831F1BBAB88002C547CF0B38BB3
:10963000B8A804285078F1B088B49726A85998BBE8
:10964000ABB38B02264666B0B8F08A9CA829517944
:109650008B2951798A2470598B2058718A44693832
:109660008B3940688A6448318B30496088F1AC009E
:109670002C547CF08CA804285078F1889726A8599F
:1096800098AC8C02264666F0899CA82951792470F2
:1096900059446938644831A98809205970AB113898
:1096A0004069A8193148608CA83C415C207C00F1DD
:1096B00087981986A86E767EA999882D557DD8B190
:1096C000B5B9A3DFDFDFAED0DFAAD0DEF2ABF8F9A9
:1096D000D9B087C4AAF1DFDFBBAFDFDFB9D8B1F102
:1096E000A3978E60DFB084F2C8F8F9D9DED89385ED
:1096F000F14AB183A308B5839A0810B79F10D8F137
:10970000B0BAAEB08AC2B2B68E9EF1FBD9F41DD803
:10971000F9D90CF1D8F8F8AD61D9AEFBD8F40CF159
:10972000D8F8F8AD19D9AEFBDFD8F416F1D8F8ADFA
:109730008D61D9F4F4ACF59C9C8DDF2BBAB6AEFAF2
:10974000F8F40BD8F1AED0F8AD51DAAEFAF8F1D8A2
:10975000B9B1B6A3839C08B9B1839AB5AAC0FD304C
:1097600083B79F10B58B93F20202D1ABDADED8F14A
:10977000B080BAABC0C3B284C1C3D8B1B9F38BA3B4
:1097800091B609B4D9ABDEB0879CB9A3DDF1B38B38
:109790008B8B8B8BB087A3A3A3A3B28BB69BF2A3B7
:1097A000A3A3A3A3A3A3A3A3A3F1B087B59AA3F3F1
:1097B0009BA3A3DCBAACDFB9A3A3A3A3A3A3A3A3D6
:1097C000A3A3A3A3A3A3A3A3D8D8D8BBB3B7F1AA39
:1097D000F9DAFFD9809AAA28B48098A720B797878A
:1097E000A86688F07951F1902C870CA78197629335
:1097F000F071716085940129517990A5F1284C6C24
:10980000870C95188578A38390284C6C886CD8F3C6
:10981000A28200F210A8921980A2F2D926D8F1886B
:10982000A84DD948D896A83980D93CD89580A83970
:10983000A68698D92CDA87A72CD8A8899519A9804B
:10984000D938D8A88939A980DA3CD8A82EA8399067
:10985000D90CD8A8953198D90CD8A809D9FFD80126
:10986000DAFFD89539A9DA26FFD890A80D8999A8EA
:1098700010809821DA2ED88999A83180DA2ED8A8BC
:1098800086963180DA2ED8A8873180DA2ED8A88241
:1098900092F34180F1D92ED8A882F31980F1D92E04
:1098A000D882ACF3C0A28022F1A62EA72EA92298BE
:1098B000A829DAACDEFFD8A2F22AF1A92E8292A85A
:1098C000F23180A696F1D900AC8C9C0C30ACDED085
:1098D000DEFFD88C9CACD010ACDE8092A2F24C8221
:1098E000A8F1CAF235F19688A6D900D8F1FF000098
:1098F0004FBB610567ACDD3F182D4454FB21E93FA8
:109900009BF681D20B73EF3F182D4454FB21F93F96
:10991000E2652F227F2B7A3C075C143326A6813C1C
:10992000BDCBF07A8807703C075C143326A6913CC7
:10993000C4EB98999999C9BF711623FEC671BCBF33
:109940006D9A74AFF2B0B3BF9AFDDE522DDEADBF9B
:109950002F6C6A2C44B4A2BF0D5555555555D53FB3
:10996000FF8300922449C23F6E204CC5CD45B73FCE
:10997000513DD0A0660DB13FEB0D76244B7BA93F46
:1099800011DA22E33AAD903F000000000000000031
:1099900050726F647563742049442072656164205D
:1099A0006173203020696E6469636174657320643B
:1099B00065766963652069732065697468657220DE
:1099C000696E636F6D70617469626C65206F72207F
:1099D000616E204D5055333035302E0D0A00000099
:1099E000009A000800000020C000000028010008C4
:1099F000C09A0008C0000020080B000044010008C5
:109A000000A24A040000000000000000010203045C
:109A10000607080901000000000000000000000027
:109A2000000000000000000000000000010203042C
:109A300001020304060708090204060800000000EA
:109A40000000000001000000000000000000000015
:109A5000000000000000000000000000B48C0008BE
:109A6000A88C0008000000000000000000000000BA
:109A700000000000000000000000000000000000E6
:109A800000000000D08C0008000000000000000072
:109A900000000000000000000000000000000000C6
:109AA0000000803F000000000000000000000000F7
:109AB000FF000000FF0000000100000000000000A7
:04000005080000ED02
:00000001FF
